:100000000C94D4020C9418030C9418030C94180349
:100010000C9418030C9418030C9418030C941803F4
:100020000C9418030C9418030C94E8160C94BA174B
:100030000C946C290C9418030C9418030C9418035A
:100040000C9418030C9418030C9418030C941803C4
:100050000C9418030C94D9290C9418030C941803CD
:100060000C9418030C9418030C9418030C941803A4
:100070000C9418030C9418030C9418030C94180394
:100080000C941C0E0C9418030C9418030C94180375
:100090000C9418030C9418030C9418030C94180374
:1000A0000C9418030C9418030C941803076342363D
:1000B000B79BD8A71A39685618AEBAAB558C1D3CF9
:1000C000B7CC5763BD6DEDFD753EF6177231BF00BD
:1000D0000000803F08000000BE922449123EABAAF7
:1000E000AA2ABECDCCCC4C3E00000080BEABAAAA52
:1000F000AA3E00000000BF000000803F000000009A
:1001000000084178D3BB4387D1133D190E3CC3BDD2
:100110004282AD2B3E68EC8276BED98FE1A93E4C7F
:1001200080EFFFBE01C4FF7F3F00000000003500EC
:100130001E001F00200021002200230024002500B3
:10014000260027002A002B0014001A0008001500C2
:1001500017001C0018000C00120013002A002900D0
:1001600004001600070009000A000B000D000E0035
:100170000F0033003400E1001D001B0006001900D1
:10018000050011001000360037003800280000304C
:10019000E000E200E30003522C002C000452500067
:1001A000510052004F0035001E001F0020002100AA
:1001B0002200230024002500260027002A002B000F
:1001C00014001A00090013000A000D000F001800A7
:1001D0001C0033002A002900040015001600170037
:1001E00007000B00110008000C0012003400E100B1
:1001F0001D001B000600190005000E00100036004F
:100200003700380028000030E000E200E30003522D
:100210002C002C0004525000510052004F003500B9
:100220001E001F00200021002200230024002500C2
:10023000260027002A002B00340036003700130068
:100240001C0009000A00060015000F002A00290002
:1002500004001200080018000C0007000B00170033
:10026000110016003800E100330014000D000E00EC
:100270001B00050010001A0019001D0028000030A6
:10028000E000E200E30003522C002C000452500076
:10029000510052004F0035001E001F0020002100B9
:1002A0002200230024002500260027002A00350212
:1002B0001E021F0220022102220223022402250222
:1002C000260227022A0001003A003B003C003D00C4
:1002D0003E003F002D022E022F02300231020100AB
:1002E00040004100420043004400450000530153D8
:1002F0000253005001000100010001000100010053
:10030000010001000100AB00AA00A900AE00350009
:100310001E001F00200021002200230024002500D1
:10032000260027002A0035001E001F0020002100A3
:100330002200230024002500260027002A000100B7
:100340003A003B003C003D003E003F002D002E00E7
:100350002F00300031000100400041004200430006
:1003600044004500005301530253005001000100B6
:100370000100010001000100010001000100AB00CB
:10038000AA00A900AE002A035400680065002000FE
:100390005000720065006F006E006900630020006D
:1003A0004B006500790062006F006100720064001C
:1003B00000002C034F007200740068006F006C0096
:1003C00069006E0065006100720020004B0065004E
:1003D000790062006F006100720064007300000029
:1003E000040309040902D000060100A0FA09040070
:1003F000000103010100092111010001223F000752
:1004000005810308000A0904010001030102000933
:100410002111010001224D000705820308000A098D
:10042000040200010300000009211101000122362D
:10043000000705830308000A090403000203000003
:10044000000921110100012220000705840320007A
:100450000107050403200001090404000001010054
:100460000009240100010900010509040500020139
:1004700003000007240100014100062402010100DD
:1004800006240202020009240301030102010009FB
:1004900024030204010101000905060240000500D1
:1004A0000005250101010905850240000500000540
:1004B000250101031201100100000008EDFE61603A
:1004C0000100010200010631FF0974A1010975153F
:1004D0000025FF9520750881020976150025FF95F6
:1004E0002075089102C005010980A101850216014D
:1004F0000026B7001A01002AB70075109501810087
:10050000C0050C0901A1018503160100269C021AF1
:1005100001002A9C02751095018100C005010902A5
:10052000A1010901A10005091901290515002501ED
:100530009505750181029501750381010501093059
:1005400009311581257F95027508810609381581C5
:10055000257F950175088106050C0A38021581254D
:100560007F950175088106C0C005010906A1010536
:100570000719E029E7150025019508750181029505
:100580000175088101050819012905950575019175
:10059000029501750391010507190029FF15002532
:1005A000FF950675088100C011241FBECFEFDAE069
:1005B000DEBFCDBF04B603FE24C080910404909139
:1005C0000504A0910604B09107048730904BA74022
:1005D000B04BB9F410920404109205041092060472
:1005E0001092070414BE84B7877F84BF88E10FB6DA
:1005F000F89480936000109260000FBEE0E0F8E392
:10060000099512E0A0E0B1E0EEE1F9E602C0059044
:100610000D92A832B107D9F714E0A8E2B2E001C008
:100620001D92A430B107E1F70E94A0130C948D3401
:100630000C94000061110DC0FC018281882331F00F
:1006400085EE0E94671E0E94683003C085EE0E94FE
:100650002F1F80E090E008950E940F0E40E050E0D0
:1006600069E070E080E091E00C94600F08950E94D2
:1006700049036E9A769A8CE293E0892B11F00C94E0
:100680002C03089586E393E0892B11F00C94360334
:100690000895279A2F988FEF9FEF9093870080936C
:1006A00086008AE08093800089E1809381000C9429
:1006B000113081110BC080918000877F8093800072
:1006C00010928D0010928C002F9808952F988330EF
:1006D00041F4809180008860809380008FEF9FEFCD
:1006E00012C09091800098609093800023E030E0E9
:1006F000281B3109220F331F8FEF9FEF02C0969501
:1007000087952A95E2F790938D0080938C00089549
:100710008B3B910568F4883A910530F5853A91054F
:10072000C0F48430910598F4019709F06FC071C04E
:10073000803E910508F46AC0883E910540F09C0116
:10074000205F31092031310508F060C05CC09C0198
:10075000A1C0853A910509F45FC0863A910509F474
:100760005EC023E830E496C0883A910509F45AC087
:10077000893A910509F459C08A3A910509F458C09B
:100780008B3A910509F457C08C3A910509F456C08B
:100790008D3A910509F455C0803B910509F454C088
:1007A0008E3A910509F453C08F3A910509F452C06D
:1007B000813B910509F451C0823B910509F450C079
:1007C000833B910509F44FC0843B910509F44EC069
:1007D000853B910509F44DC0863B910509F44CC059
:1007E000873B910509F44BC0883B910509F44AC049
:1007F000893B910509F449C08A3B910509F048C03D
:100800002AE236E447C09C01306544C020E030E075
:1008100041C021E030E03EC021E830E43BC022E8A6
:1008200030E438C022EE34E435C029EE34E432C07E
:100830002AEE34E42FC025EB34E42CC026EB34E45C
:1008400029C027EB34E426C02CEC34E423C02DEC83
:1008500034E420C023E835E41DC02AE835E41AC09A
:1008600022E935E417C024E935E414C021E236E476
:1008700011C023E236E40EC024E236E40BC025E2C8
:1008800036E408C026E236E405C027E236E402C0BA
:1008900020E034E4C90108959CE0799FF00111241F
:1008A0009CE3899FE00DF11D1124E60FF11DEE0F71
:1008B000FF1FE25DFE4F25913491C9010895880F15
:1008C000991F82559040FC0125913491C9010895EA
:1008D000880F991F825D9E4FFC0125913491C901BB
:1008E00008950E944C049C019A9581159F4110F433
:1008F000C9010895C90190528115904128F4C90198
:100900009F700E9468040895C90190538115904119
:1009100020F4C9019927906C0895C901905440971B
:1009200028F4C9018F709927946D0895203180E4CF
:10093000380719F480E091ED0895213190E43907EA
:1009400019F480E090ED0895223140E4340719F461
:1009500080E092ED0895233180E4380719F480E0B7
:1009600093ED0895211590E5390799F40E945623D7
:1009700040E065E088E491E00E94600F2FEF44E3DF
:100980008CE0215040408040E1F700C000000C9412
:10099000FE29213090E5390731F48091F002816021
:1009A0008093F0020895C90190558115904108F097
:1009B00062C0432F55274F70552741305105F9F438
:1009C000C90174E0880F991F7A95E1F78827937021
:1009D000B901E3E0660F771FEA95E1F760767727C4
:1009E000862B972B9C682370332702C0440F551F1A
:1009F0002A95E2F74F715527842B952B08954230A5
:100A0000510529F4922F8827816F906A0895433009
:100A10005105B9F4C90153E0880F991F5A95E1F7C0
:100A2000807E97702370332741E050E002C0440F6E
:100A3000551F2A95E2F74F715527842B952B9C68FB
:100A400008954430510589F5C90143E0880F991F85
:100A50004A95E1F7807E97702370332741E050E09C
:100A600002C0440F551F2A95E2F74F715527842B7A
:100A7000952B9A680895C90190568115904118F4F4
:100A8000C901906F0895C90190578115904120F4D4
:100A9000C9019F7090620895C901905881159041D5
:100AA00020F4C9019F70906A0895203E3105E0F45A
:100AB000203C310568F52133310509F475C048F44F
:100AC0002932310509F46BC02A32310509F07BC0A7
:100AD00075C02933310501F122383105E9F025339C
:100AE000310509F070C051C0233E3105B1F140F429
:100AF000203E3105D1F0223E310509F064C01CC012
:100B0000263E310579F1273E310509F05CC038C039
:100B1000C9010E945F0408958091010380FD02C015
:100B200081FF51C080EE90E04FC08091010380FFB3
:100B3000F9CF89E390E048C08091010382FF0AC0A9
:100B40008091010384FF03C080E090E03DC083EE0C
:100B500090E03AC082EE90E037C08091010382FFBE
:100B6000EFCFF8CF8091010383FF07C0809101038D
:100B700084FDEACF87EE90E027C086EE90E024C0A7
:100B80008091010383FFF2CFF8CF8091010385FFAD
:100B900003C089E290E018C085E390E015C0809121
:100BA000010385FDF9CFF5CF8091010386FF03C0D6
:100BB0008AE290E009C081E390E006C080910103E1
:100BC00086FDF9CFF5CFC9010E94880308950895E5
:100BD0005F926F927F928F929F92AF92BF92CF92CD
:100BE000DF92EF92FF920F931F93CF93DF93CDB7D6
:100BF000DEB72A970FB6F894DEBF0FBECDBF9E01B9
:100C00002F5F3F4F4E018BE0880E911C60E070E03B
:100C100000E010E0E12CF12CC12CD12CA12CB12C46
:100C20008AE0782E622E532E41E050E0E3E9F1E0B5
:100C3000A62DB52D872D01900D928A95E1F7F9012A
:100C4000819191919F01FC01E07FFF27E032F10546
:100C500059F48F709927FA0102C0EE0FFF1F8A9591
:100C6000E2F7AE2ABF2A37C0E033F10559F48F709E
:100C70009927FA0102C0EE0FFF1F8A95E2F7CE2AEC
:100C8000DF2A29C0E034F10559F48F709927FA0161
:100C900002C0EE0FFF1F8A95E2F7EE2AFF2A1BC063
:100CA000E035F10559F48F709927FA0102C0EE0F73
:100CB000FF1F8A95E2F70E2B1F2B0DC0E036F105C2
:100CC00051F48F709927FA0102C0EE0FFF1F8A9529
:100CD000E2F76E2B7F2B2815390509F0A7CF94B1C9
:100CE0008A2D8095892384B985B18A2985B997B1E0
:100CF0008C2D8095892387B988B18C2988B99AB1C0
:100D00008E2D809589238AB98BB18E298BB99DB19F
:100D1000802F809589238DB98EB1802B8EB990B3A9
:100D2000862F8095892380BB81B3862B81BB2A9631
:100D30000FB6F894DEBF0FBECDBFDF91CF911F91EC
:100D40000F91FF90EF90DF90CF90BF90AF909F906A
:100D50008F907F906F905F9008955F926F927F92D7
:100D60008F929F92AF92BF92CF92DF92EF92FF92BB
:100D70000F931F93CF93DF93CDB7DEB768970FB66E
:100D8000F894DEBF0FBECDBF85B7806885BF85B73D
:100D9000806885BF0E94E8059E012F5F3F4F4E018E
:100DA00089E1880E911C60E070E000E010E0E12C29
:100DB000F12CC12CD12CA12CB12C98E1792E622ED2
:100DC000532E41E050E0EDE9F1E0A62DB52D872D41
:100DD00001900D928A95E1F7F901819191919F011E
:100DE000FC01E07FFF27E032F10559F48F7099276D
:100DF000FA0102C0EE0FFF1F8A95E2F7AE2ABF2A62
:100E000037C0E033F10559F48F709927FA0102C019
:100E1000EE0FFF1F8A95E2F7CE2ADF2A29C0E034C1
:100E2000F10559F48F709927FA0102C0EE0FFF1FE8
:100E30008A95E2F7EE2AFF2A1BC0E035F10559F446
:100E40008F709927FA0102C0EE0FFF1F8A95E2F713
:100E50000E2B1F2B0DC0E036F10551F48F70992732
:100E6000FA0102C0EE0FFF1F8A95E2F76E2B7F2B6F
:100E70002815390509F0A7CF94B18A2D80958923CB
:100E800084B985B18A2985B997B18C2D809589233C
:100E900087B988B18C2988B99AB18E2D809589231C
:100EA0008AB98BB18E298BB99DB1802F809589230A
:100EB0008DB98EB1802B8EB990B3862F8095892302
:100EC00080BB81B3862B81BB10922902109228022D
:100ED000109233021092320210922B0210922A02C8
:100EE000109235021092340210922D0210922C02B0
:100EF000109237021092360210922F0210922E0298
:100F0000109239021092380210923102109230027F
:100F100010923B0210923A0287E393E0892BB9F0DA
:100F200068960FB6F894DEBF0FBECDBFDF91CF91AC
:100F30001F910F91FF90EF90DF90CF90BF90AF90F7
:100F40009F908F907F906F905F900C94370368967E
:100F50000FB6F894DEBF0FBECDBFDF91CF911F91CA
:100F60000F91FF90EF90DF90CF90BF90AF909F9048
:100F70008F907F906F905F9008955F926F927F92B5
:100F80008F929F92AF92BF92CF92DF92EF92FF9299
:100F90000F931F93CF93DF93CDB7DEB7A2970FB612
:100FA000F894DEBF0FBECDBF7E0149E1E40EF11C17
:100FB00022E3C22E22E0D22E5E0153E2A50EB11C26
:100FC0003AE0532E470101E010E048E1642E55E07D
:100FD000752EE3E9F1E0D401852D01900D928A95FB
:100FE000E1F7F701819191917F019C01207F3327E7
:100FF0002032310589F424B18F709927A80102C0ED
:10100000440F551F8A95E2F7CA01242B24B995B1E4
:101010008095892385B94FC02033310589F427B1E4
:101020008F709927F80102C0EE0FFF1F8A95E2F733
:10103000CF012E2B27B998B18095892388B93BC061
:101040002034310589F42AB18F709927A80102C094
:10105000440F551F8A95E2F7CA01242B2AB99BB188
:10106000809589238BB927C02035310589F42DB1AE
:101070008F709927F80102C0EE0FFF1F8A95E2F7E3
:10108000CF012E2B2DB99EB1809589238EB913C027
:101090002036310581F420B38F709927A80102C052
:1010A000440F551F8A95E2F7CA01242B20BB91B348
:1010B0008095892381BB50EA5A95F1F7BE016F5F95
:1010C0007F4F80E090E020E030E0EDE9F1E0DE01EC
:1010D0001196462D01900D924A95E1F7FB01419141
:1010E0005191BF01FA01E07FFF27E032F10511F4D1
:1010F000E3B113C0E033F10511F4E6B10EC0E03402
:10110000F10511F4E9B109C0E035F10511F4ECB1D4
:1011100004C0E036F105B9F4EFB1F0E04F705527A7
:1011200002C0F595E7954A95E2F7E0FD08C0A801F1
:10113000022E02C0440F551F0A94E2F702C040E09D
:1011400050E0842B952B2F5F3F4F2C30310509F059
:10115000BCCFF601208131812817390721F0918316
:101160008083709270010E94E805F2E0CF0ED11CDE
:10117000EA14FB0409F02DCF809170018823A1F1BE
:10118000815080937001882339F08FE99FE00197A7
:10119000F1F700C0000028C0809132029091330224
:1011A0009093290280932802809134029091350215
:1011B00090932B0280932A028091360290913702FD
:1011C00090932D0280932C028091380290913902E5
:1011D00090932F0280932E0280913A0290913B02CD
:1011E000909331028093300282E493E0892B11F0D6
:1011F0000E94420381E0A2960FB6F894DEBF0FBEB4
:10120000CDBFDF91CF911F910F91FF90EF90DF90B5
:10121000CF90BF90AF909F908F907F906F905F9096
:101220000895E82FF0E0EE0FFF1FE85DFD4F80818D
:10123000918108950895CF92DF92EF92FF920F93DC
:101240001F93CF93DF93CDB7DEB7CC5BD2400FB601
:10125000F894DEBF0FBECDBF8C01862F642F88238C
:1012600079F0F80192812FE7482F992329F083E044
:1012700093E00E94C41904C083E093E00E94D41953
:10128000F80180818B3091F59181943009F0A8C2EA
:101290009281809173019923B1F08F5F80937301E4
:1012A00096E4E5EBF1E0DE01A958BD4F01900D9207
:1012B0009A95E1F7E0917101F0917201EE0FFF1F35
:1012C00027E732E036C096E4E5EBF1E0DE01AF5C03
:1012D000BD4F01900D929A95E1F7E0917101F09167
:1012E0007201EE0FFF1F21E332E093C08A3009F054
:1012F000CBC0F8019181943009F072C29281809143
:101300007301992309F473C081508093730196E4AB
:10131000E5EBF1E0DE01A551BE4F01900D929A95EB
:10132000E1F7E0917101F0917201EE0FFF1F2BEEDA
:1013300031E02C0F3D1FE20FF31F60817181680FB8
:10134000711D882777FD8095982F0E94AC3120E091
:1013500030E040E451E40E94113120E030E040E808
:1013600050E40E94A9309B01AC0160E070E080E095
:1013700090E40E94C33221E230ED42E053E40E9447
:1013800060324CE050E00E94BB0F20E04BE760E091
:1013900083E093E00E94B41920E04BE761E083E032
:1013A00093E00E94B41920E04BE762E083E093E011
:1013B0000E94B41920E04BE763E083E093E00E94D1
:1013C000B41920E04BE764E083E093E0C454DD4FC0
:1013D0000FB6F894DEBF0FBECDBFDF91CF911F9146
:1013E0000F91FF90EF90DF90CF900C94B41996E49A
:1013F000E5EBF1E0DE01AB55BE4F01900D929A9501
:10140000E1F7E0917101F0917201EE0FFF1F25EA03
:1014100031E02C0F3D1FE20FF31F60817181680FD7
:10142000711D882777FD8095982F0E94AC3120E0B0
:1014300030E040E451E40E94113120E030E040E827
:1014400050E40E94A9309B01AC0160E070E080E0B4
:1014500090E40E94C33221E230ED42E053E40E9466
:1014600060320E94EB0CC454DD4F0FB6F894DEBF1F
:101470000FBECDBFDF91CF911F910F91FF90EF90E5
:10148000DF90CF900C94BE0C893009F0D3C0F801E6
:101490009181943009F0A4C19281992309F4A0C1EB
:1014A00080917101909172010196909372018093E5
:1014B000710120E04BE760E083E093E00E94B41903
:1014C00020E04BE761E083E093E00E94B41920E064
:1014D0004BE762E083E093E00E94B41920E04BE721
:1014E00063E083E093E00E94B41920E04BE764E0FE
:1014F00083E093E00E94B4190E94BE0C00E010E06B
:10150000E6E4FE2E80917301E5EBF1E0DE01A15AE5
:10151000BE4F9F2D01900D929A95E1F7E0917101D8
:10152000F0917201E00FF11FEE0FFF1F2FE531E088
:101530002C0F3D1FE20FF31F60817181680F711D39
:10154000882777FD8095982F0E94AC3120E030E00D
:1015500040E451E40E94113120E030E040E850E4E2
:101560000E94A9309B01AC0160E070E080E090E453
:101570000E94C33221E230ED42E053E40E94603227
:101580004CE050E00E94BB0F3FEF87EE93E03150FC
:1015900080409040E1F700C0000080917301E5EBCE
:1015A000F1E0DE01A75EBE4F9F2D01900D929A954E
:1015B000E1F7E0917101F0917201E00FF11FEE0F80
:1015C000FF1F29E131E02C0F3D1FE20FF31F608167
:1015D0007181680F711D882777FD8095982F0E9473
:1015E000AC3120E030E040E451E40E94113120E0D1
:1015F00030E040E850E40E94A9309B01AC0160E07B
:1016000070E080E090E40E94C33221E230ED42E0DD
:1016100053E40E9460320E94EB0C8FEF9CE701972D
:10162000F1F700C000000F5F1F4F0830110509F0EF
:1016300069CF94C1883009F0D3C0F801918194300A
:1016400009F0CEC09281992309F4CAC0809171013A
:10165000909172010197909372018093710120E043
:101660004BE760E083E093E00E94B41920E04BE791
:1016700061E083E093E00E94B41920E04BE762E070
:1016800083E093E00E94B41920E04BE763E083E03D
:1016900093E00E94B41920E04BE764E083E093E01C
:1016A0000E94B4190E94BE0C00E010E056E4F52E32
:1016B00080917301E5EBF1E0DE01AD52BF4F9F2D4C
:1016C00001900D929A95E1F7E0917101F09172010C
:1016D000E00FF11FEE0FFF1F23ED30E02C0F3D1F39
:1016E000E20FF31F60817181680F711D882777FDFC
:1016F0008095982F0E94AC3120E030E040E451E426
:101700000E94113120E030E040E850E40E94A9300E
:101710009B01AC0160E070E080E090E40E94C33285
:1017200021E230ED42E053E40E9460324CE050E0B0
:101730000E94BB0F3FEF87EE93E031508040904016
:10174000E1F700C0000080917301E5EBF1E0DE01FC
:10175000A357BF4F9F2D01900D929A95E1F7E0910D
:101760007101F0917201E00FF11FEE0FFF1F2DE8E4
:1017700030E02C0F3D1FE20FF31F60817181680F75
:10178000711D882777FD8095982F0E94AC3120E04D
:1017900030E040E451E40E94113120E030E040E8C4
:1017A00050E40E94A9309B01AC0160E070E080E051
:1017B00090E40E94C33221E230ED42E053E40E9403
:1017C00060320E94EB0C8FEF9CE70197F1F700C0AD
:1017D00000000F5F1F4F0830110509F069CFBEC030
:1017E000F801228190917301222309F45DC026E45F
:1017F000E5EBF1E0DE01A95BBF4F01900D922A9568
:10180000E1F7E0917101F0917201E80FF11DEE0F27
:10181000FF1F27E430E02C0F3D1FE20FF31F608114
:101820007181690F711D882777FD8095982F0E941F
:10183000AC3120E030E040E451E40E9411316B0112
:101840007C01F801818165E070E0681B71098827DF
:1018500077FD8095982F0E94AC319B01AC01C701A8
:10186000B6010E94A9309B01AC0160E070E080E00D
:1018700090E40E94C33221E230ED42E053E40E9442
:1018800060324FE050E0C454DD4F0FB6F894DEBF35
:101890000FBECDBFDF91CF911F910F91FF90EF90C1
:1018A000DF90CF900C94BB0F26E4E5EBF1E0DE0176
:1018B000119601900D922A95E1F7E0917101F09156
:1018C0007201E80FF11DEE0FFF1F21E030E02C0F39
:1018D0003D1FE20FF31F60817181690F711D882721
:1018E00077FD8095982F0E94AC3120E030E040E4F5
:1018F00051E40E9411316B017C01F801818165E0A6
:1019000070E0681B7109882777FD8095982F0E94E9
:10191000AC319B01AC01C701B6010E94A9309B010B
:10192000AC0160E070E080E090E40E94C33221E20C
:1019300030ED42E053E40E946032C454DD4F0FB6F4
:10194000F894DEBF0FBECDBFDF91CF911F910F91F5
:10195000FF90EF90DF90CF900C94EB0CC454DD4FD0
:101960000FB6F894DEBF0FBECDBFDF91CF911F91B0
:101970000F91FF90EF90DF90CF9008951092870223
:1019800010928602809171008D7F8093710080910A
:1019900090008F7780939000109248021092470237
:1019A00010928002109281021092820210928302A1
:1019B00010927F0210927E02EEE5F2E0AEE4B2E019
:1019C00011921192119211921D921D9282E0EE37A6
:1019D000F807B1F708956F927F928F929F92AF921E
:1019E000BF92CF92DF92EF92FF920F931F93CF930C
:1019F000DF936B017C010EE712E04CE5A42E42E080
:101A0000B42EC7E0D0E0A7019601F801929182912F
:101A1000729162918F010E940D31882349F02197C4
:101A2000F2E0AF1AB108CF3F8FEFD80761F734C0AB
:101A3000F8011082118212821382F5011182108244
:101A4000FE01EE0FFF1FEE0FFF1FE25AFD4FDE01FA
:101A5000AA0FBB1FA25BBD4FCE011AC001964481E5
:101A600055816681778140835183628373831482B9
:101A700015821682178212962D913C91139711961A
:101A80003C932E9313961C921E92129734961296A4
:101A90008730910519F7C3CF809186029091870214
:101AA000019797FD05C0909387028093860204C03A
:101AB0001092870210928602E0918602F0918702CE
:101AC0003097C9F4809171008D7F8093710080916F
:101AD00090008F7780939000109280021092810284
:101AE000109282021092830210927F0210927E0264
:101AF0001092470285C03197DF01AA0FBB1FAA0FC2
:101B0000BB1FA25ABD4FCD90DD90ED90FC90EE0F23
:101B1000FF1FE25BFD4FC081D18160908002709019
:101B200081028090820290908302A7019601662D27
:101B3000772D882D992D0E940D3187FF25C0262DE8
:101B4000372D482D592DC701B6010E94A83020E03D
:101B500030E04AEF54E40E9411315B018C012A2DE0
:101B60003B2D402F512F662D772D882D992D0E94CA
:101B7000A9303B014C01A7019601772D992D0E94B8
:101B80000D31181664F72EC0A7019601662D772D2A
:101B9000882D992D0E945C32181634F5A701960104
:101BA000662D772D882D992D0E94A83020E030E0F9
:101BB0004AEF54E40E9411315B018C012A2D3B2D28
:101BC000402F512F662D772D882D992D0E94A830FA
:101BD0003B014C01A7019601772D992D0E945C32A3
:101BE00087FFECCF10924D02C0928002D09281020A
:101BF000E0928202F0928302D0937F02C0937E0231
:101C0000DF91CF911F910F91FF90EF90DF90CF90D8
:101C1000BF90AF909F908F907F906F9008953E9A65
:101C2000E1E7F0E080818D7F808382E08093900007
:101C30008AE18093910008951F920F920FB60F9240
:101C40001124CF92DF92EF92FF922F933F934F9305
:101C50005F936F937F938F939F93AF93BF93CF9334
:101C6000DF93EF93FF9380914702882309F479C0B3
:101C700020E030E0A90160918002709181028091A2
:101C80008202909183020E945C3218160CF069C0A7
:101C900020E030E040E251E46091490270914A0254
:101CA00080914B0290914C020E945C321816BCF459
:101CB00080918402909185020196609186027091D4
:101CC00087020E9448349093850280938402109288
:101CD000490210924A0210924B0210924C02C0919B
:101CE0008402D0918502CC0FDD1FCC0FDD1FC25ABC
:101CF000DD4F288139814A815B8160E074E284E7AD
:101D00009BE40E9411310E94793170939700609397
:101D10009600288139814A815B8160E074E284E722
:101D20009BE40E9411310E947931759567957093FB
:101D300099006093980020E030E040E85FE3609114
:101D4000490270914A0280914B0290914C020E948C
:101D5000A9306093490270934A0280934B0290939A
:101D60004C0280914802882309F493C0C09043023A
:101D7000D0904402E0904502F090460220E030E02E
:101D8000A901C701B6010E945C321816F4F4A7013C
:101D9000960160E074E284E79BE40E9411310E94A6
:101DA00079317093970060939600A701960160E0E7
:101DB00074E284E79BE40E9411310E9479317595A9
:101DC0006795709399006093980060913D027091BF
:101DD0003E026F5F7F4F70933E0260933D0280E052
:101DE00090E00E94AA3120913F0230914002409140
:101DF0004102509142020E945C3287FD4AC08091AC
:101E00003C028F5F80933C029091F0038917A0F011
:101E10008091F503882319F010923C020DC0809147
:101E200071008D7F80937100809190008F778093F7
:101E30009000109248022DC0E091F103F091F2035E
:101E400080913C0298E0899FE00DF11D1124808172
:101E50009181A281B3818093430290934402A09325
:101E60004502B093460220E030E040E85EE3648142
:101E70007581868197810E94603260933F027093E2
:101E80004002809341029093420210923E021092CF
:101E90003D02FF91EF91DF91CF91BF91AF919F9163
:101EA0008F917F916F915F914F913F912F91FF9013
:101EB000EF90DF90CF900F900FBE0F901F9018956E
:101EC0000F931F93CF93DF9300D0CDB7DEB78C0174
:101ED00080914702882331F04A8369830E94BE0CB7
:101EE00069814A8181E0809348021093F203009354
:101EF000F1036093F0034093F503109249021092AE
:101F00004A0210924B0210924C0210923C02F801CD
:101F10004081518162817381409343025093440216
:101F2000609345027093460220E030E040E85EE3B3
:101F300064817581868197810E94603260933F023F
:101F400070934002809341029093420210923E02AD
:101F500010923D02809171008260809371008091A7
:101F600090008068809390000F900F90DF91CF9148
:101F70001F910F9108956F927F928F929F92AF92CF
:101F8000BF92CF92DF92EF92FF920F931F93CF9366
:101F9000DF936B017C01EA018091480281110E946C
:101FA000BE0C81E08093470220E030E0A901C70128
:101FB000B6010E945C3218160CF09AC06090800244
:101FC00070908102809082029090830220E030E045
:101FD000A901662D772D882D992D0E940D31811133
:101FE00028C0C0928002D0928102E0928202F092D8
:101FF0008302D0937F02C0937E02809186029091EB
:102000008702FC01EE0FFF1FEE0FFF1FE25AFD4F8C
:10201000C082D182E282F382FC01EE0FFF1FE25BFD
:10202000FD4FD183C08301969093870280938602EF
:102030005FC0A7019601662D772D882D992D0E94EE
:102040000D3187FF25C0262D372D482D592DC7016D
:10205000B6010E94A83020E030E04AEF54E40E942C
:1020600011315B018C012A2D3B2D402F512F662D04
:10207000772D882D992D0E94A9303B014C01A70195
:102080009601772D992D0E940D31181664F7A9CF6E
:10209000A7019601662D772D882D992D0E945C321F
:1020A00018160CF09ECFA7019601662D772D882D6E
:1020B000992D0E94A83020E030E04AEF54E40E94BD
:1020C00011315B018C012A2D3B2D402F512F662DA4
:1020D000772D882D992D0E94A8303B014C01A70136
:1020E0009601772D992D0E945C3287FFECCF79CF36
:1020F000809171008260809371008091900080686F
:1021000080939000DF91CF911F910F91FF90EF90FE
:10211000DF90CF90BF90AF909F908F907F906F9007
:102120000895809191020895CF93DF9300D01F927C
:10213000CDB7DEB72091FA03243021F523E02983BF
:102140009B838A832093E9008FEF06C095ED9A95D3
:10215000F1F70000882329F09091E800815095FF65
:10216000F5CF8091E80085FF0DC040E050E063E0CE
:1021700070E0CE0101960E947E148091E8008E7777
:102180008093E8000F900F900F90DF91CF9108950A
:10219000CF93DF9300D01F92CDB7DEB72091FA0323
:1021A000243029F522E029839B838A8383E080936E
:1021B000E9008FEF06C095ED9A95F1F700008823AE
:1021C00029F09091E800815095FFF5CF8091E800CB
:1021D00085FF0DC040E050E063E070E0CE01019665
:1021E0000E947E148091E8008E778093E8000F9023
:1021F0000F900F90DF91CF9108952091FA03243032
:10220000F9F422E02093E9002FEF06C035ED3A956E
:10221000F1F70000222329F03091E800215035FF2A
:10222000F5CF2091E80025FF0BC040E050E065E0CD
:1022300070E00E947E148091E8008E778093E80021
:102240000895CF93DF93EC018091FA03843041F538
:1022500081E08093E9008FEF06C095ED9A95F1F744
:102260000000882329F09091E800815095FFF5CF78
:102270008091E80085FF14C040E050E068E070E025
:10228000CE010E947E148091E8008E778093E80052
:1022900088E0FE01A9E8B2E001900D928A95E1F78D
:1022A000DF91CF910895BF92CF92DF92EF92FF928C
:1022B0000F931F93CF93DF937C01B62EE90100E0CB
:1022C00010E0C42ED12C0BC04991202F2B0D2F775D
:1022D0004F776FE0C7010E94B4190F5F1F4F0C15B5
:1022E0001D0594F3DF91CF911F910F91FF90EF9017
:1022F000DF90CF90BF90089570E06F5F7F4F6F7059
:1023000077270C94B4190F931F93CF93C42F633086
:10231000710509F04AC0842F807F803849F18039E7
:1023200009F043C0622F6F7770E080E090E00E9478
:10233000AC3120E030E040E451E40E9411319B01D7
:10234000AC0160E070E080E090E40E94C3320F775F
:1023500010E023E0159507952A95E1F72DEC3CEC6C
:1023600042E053E40E946032A8010E94BB0F1DC0EE
:10237000622F6F7770E080E090E00E94AC3120E047
:1023800030E040E451E40E9411319B01AC0160E077
:1023900070E080E090E40E94C3322DEC3CEC42E01F
:1023A00053E40E9460320E94EB0CCC3F29F4CF91A1
:1023B0001F910F910C94BE0CCF911F910F91089516
:1023C0000F931F93CF93DF93CDB7DEB727970FB649
:1023D000F894DEBF0FBECDBF8C0114C08A810E946D
:1023E0008E199A819D839B819E839C819F838111FD
:1023F0001EC089818430B1F08730A1F08630A1F011
:102400008530A1F0BE016F5F7F4F84E791E00E94AD
:10241000FB1C8111E3CF84E791E00E94EC1C0E9439
:1024200067190DC083E003C082E001C081E0AE0106
:102430004B5F5F4F682FC8010E94211AE3CF279698
:102440000FB6F894DEBF0FBECDBFDF91CF911F91C5
:102450000F910895EF92FF920F93CF93DF9300D0E7
:1024600000D000D0CDB7DEB77B014A832B830C832D
:10247000842F2E834D830E948E192E814D818111D0
:102480001BC082E0E816F10479F083E0E816F1045D
:1024900021F0EA94EF2821F50BC0073F11F487E003
:1024A00001C084E089830BC0273FD9F786E0FACFCB
:1024B000473FB9F785E0F6CF42954F704983BE019B
:1024C0006F5F7F4F84E791E00E94B11C84E791E049
:1024D0000E94CF1C84E791E00E94EC1C0E946719C7
:1024E00026960FB6F894DEBF0FBECDBFDF91CF9119
:1024F0000F91FF90EF9008958091F903811109C029
:102500000E946D160E94CA168091E200846080933A
:10251000E20008951092F9030895089508950C9427
:102520006129809192028F5F8093920262E30E9400
:102530002834911135C01092920280919302882321
:1025400079F18091FA03843049F58091E9008F7028
:102550009091EC0090FF02C090E801C090E0982BB1
:1025600084E08093E9008091EB0080FF14C08091AB
:10257000EE0087FD03C00FC01092F1008091E800CB
:1025800085FDFACF8091E80080FF05C08091E800CA
:102590008E778093E8009F709093E90010929302E9
:1025A000089542E061EC81E00E94E31542E061ECB5
:1025B00082E00E94E31542E061EC83E00E94E315B3
:1025C00042E261EC84E00E94E31542E361E885E0C9
:1025D0000E94E31542E360E886E00C94E3158091E5
:1025E000FC03833009F454C030F4813071F0823040
:1025F00009F0A5C08CC08A3009F479C08B3009F489
:102600005FC0893009F09BC020C08091FB03813AF4
:1026100009F095C08091E800877F8093E800809161
:10262000FF0390910004892B21F060E080E090E0AE
:1026300003C068E089E892E070E00E941C15809178
:10264000E8008B778093E80008958091FB03813246
:1026500009F075C08091FF0390910004892B09F067
:102660006EC08091E800877F8093E80005C080916C
:10267000FA03882309F463C08091E80082FFF7CF52
:102680008091F100809391028091E8008B7753C094
:102690008091FB03813A09F052C08091FF03909131
:1026A0000004892B09F04BC08091E800877F80935C
:1026B000E8008091E80080FFFCCF80918A0136C05D
:1026C0008091FB038132D9F58091FF039091000442
:1026D000892BA9F58091E800877F8093E8000E940C
:1026E0001A168091FD0380938A010C9456238091E1
:1026F000FB03813221F58091E800877F8093E80019
:102700000E941A168091FE0380938802089580919A
:10271000FB03813AA1F48091E800877F8093E80071
:102720008091E80080FFFCCF809188028093F100C7
:102730008091E8008E778093E8000C941A16089533
:1027400083E093E00E94F0196AE272E183E093E093
:102750000E94461A60EE71E183E093E00E944A1AFB
:1027600084B7877F84BF88E10FB6F89480936000B8
:10277000109260000FBE90E080E80FB6F89480934E
:102780006100909361000FBE0E94741D0E946D163F
:102790000E94CA168091E20084608093E2007894DF
:1027A00063E871E183E093E00E94EC196CE771E16A
:1027B00083E093E00E94E41963E571E183E093E034
:1027C0000E94E8190E940F0E0E9467190E94761D50
:1027D00080E891E00E94201D0BC00E941E2980917C
:1027E000F803882329F00E94492981110E94681466
:1027F0008091FA03853089F383E093E00E94F91B0E
:102800000E94801DF5CF292F332723303105B1F0E9
:102810004CF42130310509F44DC02230310509F066
:102820004EC007C02132310541F12232310591F10C
:1028300046C0E0EDF0E084EE93E045C0992781309A
:10284000910569F08230910589F0892B09F037C034
:10285000E0EEF3E0E491F0E080EE93E034C0E2EBF0
:10286000F3E0E491F0E082EB93E02DC0E6E8F3E0E2
:10287000E491F0E086E893E026C0643000F5E62FAE
:10288000F0E0EE0FFF1FE550FE4F80819181E9E0FF
:10289000F0E019C0643098F4E62FF0E0DF01AA0FF1
:1028A000BB1FAD5FBD4F8D919C91E55FFD4FE081FA
:1028B000F0E009C0E2E1F0E084EB94E004C0E0E085
:1028C000F0E080E090E0DA018D939C93CF010895D1
:1028D00080E189BD82E189BD09B400FEFDCF809110
:1028E000D8008F7D8093D8008091E0008260809333
:1028F000E0008091E00081FDFCCF0895BF92CF926F
:10290000DF92EF92FF920F931F93CF93DF937C019F
:102910008B01EA010E943B16B82E811133C020972B
:1029200031F028813981021B130BE20EF31EC12CFA
:10293000D12C23C08091E80085FD15C08091E8006E
:102940008E778093E800209749F0888199818C0DDB
:102950009D1D9983888325E0B22E14C00E943B16EA
:10296000882359F00EC0F70181917F018093F10017
:1029700001501109FFEFCF1ADF0A01151105D1F639
:1029800001C0B82E8B2DDF91CF911F910F91FF9039
:10299000EF90DF90CF90BF900895BF92CF92DF92DB
:1029A000EF92FF920F931F93CF93DF937C018B01E4
:1029B000EA010E943B16B82E811133C0209731F0F6
:1029C00028813981021B130BE20EF31EC12CD12C7E
:1029D00023C08091E80085FD15C08091E8008B77C9
:1029E0008093E800209749F0888199818C0D9D1D86
:1029F0009983888345E0B42E14C00E943B16882337
:102A000059F00EC08091F100F70181937F010150D0
:102A10001109FFEFCF1ADF0A01151105D1F601C028
:102A2000B82E8B2DDF91CF911F910F91FF90EF90DA
:102A3000DF90CF90BF90089540910104509102041F
:102A40004617570748F06115710539F44091E800C1
:102A50004E774093E80001C0BA01FC0140E033C06A
:102A60008091FA03882309F444C0853009F443C0F7
:102A70008091E80083FD41C08091E80082FD33C071
:102A80008091E80080FF1FC09091F3008091F200D8
:102A9000392F20E0A901482BCA0106C0419140937B
:102AA000F1006150710901966115710519F08830C6
:102AB0009105A0F341E0089709F040E08091E8001B
:102AC0008E778093E8006115710551F64111C8CFEA
:102AD0000AC08091FA03882361F0853061F080910B
:102AE000E80083FD0AC08091E80082FFF2CF80E019
:102AF000089582E0089583E0089581E0089540916B
:102B00000104509102044617570748F061157105FA
:102B100039F44091E8004E774093E80001C0BA01D3
:102B2000FC0140E034C08091FA03882309F445C0D9
:102B3000853009F444C08091E80083FD42C0809153
:102B4000E80082FD34C08091E80080FF20C09091B1
:102B5000F3008091F200392F20E0A901482BCA012F
:102B600007C044914093F10031966150710901967C
:102B70006115710519F08830910598F341E00897C7
:102B800009F040E08091E8008E778093E8006115BD
:102B9000710549F64111C7CF0AC08091FA03882315
:102BA00061F0853061F08091E80083FD0AC080917A
:102BB000E80082FFF2CF80E0089582E0089583E08C
:102BC000089581E00895982F2CC09093E9009817FC
:102BD00039F07091EC002091ED005091F00003C0AD
:102BE000242F762F50E021FD02C09F5F1AC0309144
:102BF000EB003E7F3093EB003091ED003D7F309352
:102C0000ED003091EB0031603093EB007093EC00FD
:102C10002093ED005093F0002091EE0027FDE5CFCA
:102C200007C0973090F28F708093E90081E008959B
:102C300080E008958091FB0387FD05C08091E80046
:102C400080FF0EC012C08091E80082FD05C0809117
:102C5000FA038111F8CF08958091E8008B7708C0BE
:102C60008091FA038111EACF08958091E8008E7770
:102C70008093E80008958091E4009091E50045E696
:102C80002091EC0020FD1FC023C02091FA032223D5
:102C900091F0253091F02091EB0025FD10C020919E
:102CA000E4003091E5002817390751F34150C9017C
:102CB00039F784E0089582E0089583E0089581E083
:102CC000089580E008952091E80020FFDECFF9CF3D
:102CD0002091E80022FFD9CFF4CF0E94DB160E949A
:102CE000E316E0EEF0E0808181608083E8EDF0E0C3
:102CF00080818F77808319BCA7EDB0E08C918E7FA7
:102D00008C9380818F7E80831092F90308950F93B6
:102D10001F93CF93DF930E94DB160E94E316C8ED4A
:102D2000D0E088818F7788838881806888838881D4
:102D30008F7D888319BC1092FA031092F6031092CB
:102D4000F8031092F70300EE10E0F80180818B7F0A
:102D5000808388818160888342E060E080E00E9417
:102D6000E315E1EEF0E080818E7F8083E2EEF0E01B
:102D7000808181608083808188608083F801808188
:102D80008E7F8083888180618883DF91CF911F91BE
:102D90000F910895E8EDF0E080818F7E8083E7ED6C
:102DA000F0E080818160808384E082BF81E0809355
:102DB000F9030C948716E8EDF0E080818E7F808324
:102DC0001092E20008951092DA001092E100089546
:102DD0001F920F920FB60F9211242F933F934F9390
:102DE0005F936F937F938F939F93AF93BF93EF9373
:102DF000FF938091E10082FF0BC08091E20082FF8F
:102E000007C08091E1008B7F8093E1000E949112C6
:102E10008091DA0080FF1FC08091D80080FF1BC026
:102E20008091DA008E7F8093DA008091D90080FF54
:102E30000DC080E189BD82E189BD09B400FEFDCFEE
:102E400081E08093FA030E947C1205C019BC1092A5
:102E5000FA030E948A128091E10080FF19C08091DC
:102E6000E20080FF15C08091E2008E7F8093E20037
:102E70008091E20080618093E2008091D8008062BE
:102E80008093D80019BC85E08093FA030E948E12CB
:102E90008091E10084FF30C08091E20084FF2CC06B
:102EA00080E189BD82E189BD09B400FEFDCF80913A
:102EB000D8008F7D8093D8008091E1008F7E809331
:102EC000E1008091E2008F7E8093E2008091E20039
:102ED00081608093E2008091F603882311F084E002
:102EE00007C08091E30087FF02C083E001C081E05A
:102EF0008093FA030E948F128091E10083FF29C022
:102F00008091E20083FF25C08091E100877F80935C
:102F1000E10082E08093FA031092F6038091E100D1
:102F20008E7F8093E1008091E2008E7F8093E200AB
:102F30008091E20080618093E20042E060E080E006
:102F40000E94E3158091F00088608093F0000E9459
:102F50008D12FF91EF91BF91AF919F918F917F91D2
:102F60006F915F914F913F912F910F900FBE0F90F6
:102F70001F9018951F920F920FB60F9211242F9346
:102F80003F934F935F936F937F938F939F93AF93F1
:102F9000BF93CF93EF93FF938091E9008F7090914F
:102FA000EC0090FF02C090E801C090E0C92FC82B50
:102FB0001092E9008091F000877F8093F000789470
:102FC0000E94FE171092E9008091F00088608093C3
:102FD000F000CF70C093E900FF91EF91CF91BF91C6
:102FE000AF919F918F917F916F915F914F913F91A1
:102FF0002F910F900FBE0F901F9018951F93CF9396
:10300000DF93CDB7DEB7AC970FB6F894DEBF0FBE37
:10301000CDBFEBEFF3E08091F100819324E0E3304A
:10302000F207C9F70E94EF128091E80083FF37C1D1
:103030008091FB039091FC03953009F488C038F42B
:103040009130B1F170F0933009F029C131C098305E
:1030500009F4F8C0993009F404C1963009F01FC191
:103060009DC0803821F0823809F019C108C08091D4
:10307000F7039091F803992389F082600FC0809143
:10308000FF03909100048F7099278093E90080914D
:10309000EB0085FB882780F91092E9009091E80009
:1030A000977F9093E8008093F1001092F100D5C0D3
:1030B000882319F0823009F0F2C08F7121F082303C
:1030C00009F0EDC00BC08091FD03813009F0E7C02D
:1030D000933009F080E08093F8032FC08091FD03C6
:1030E00081112BC08091FF03909100048F7099276C
:1030F000009709F4D4C08093E9002091EB0020FFF1
:103100001CC02091FC03233021F48091EB008062ED
:1031100012C09091EB0090619093EB0021E030E0C1
:1031200001C0220F8A95EAF72093EA001092EA0084
:103130008091EB0088608093EB001092E900809111
:10314000E800877F8093E8000E941A16A8C08111CA
:10315000A6C08091FD039091FE038F779927182FC9
:103160009091E3009078982B9093E3008091E80091
:10317000877F8093E8000E941A168091E80080FF04
:10318000FCCF8091E30080688093E300112311F06D
:1031900083E001C082E08093FA0381C080588230CE
:1031A00008F07DC08091FD039091FE038C3D23E0EB
:1031B000920779F583E08A838AE289834FB7F8948E
:1031C000DE01139620E03EE051E2E32FF0E0509361
:1031D0005700E49120FF03C0E295EF703F5FEF706E
:1031E0008E2F90E0EA3010F0C79601C0C0968D9304
:1031F0009D932F5F243149F74FBF8091E800877F6F
:103200008093E8006AE270E0CE0101960E941C15EE
:1032100013C0AE01455D5F4F6091FF030E94031430
:103220000097E9F12091E800277F2093E800BC0196
:103230008BA59CA50E947F158091E8008B778093D9
:10324000E8002DC0803859F58091E800877F809391
:10325000E8008091F6038093F1008091E8008E777A
:1032600071CF81111CC09091FD039230C0F4809108
:10327000E800877F8093E8009093F6030E941A1677
:103280008091F603811104C08091E30087FF02C0A2
:1032900084E001C081E08093FA030E94D112809102
:1032A000E80083FF0AC08091E800877F8093E800F0
:1032B0008091EB0080628093EB00AC960FB6F8949F
:1032C000DEBF0FBECDBFDF91CF911F910895CF9389
:1032D0008091FA038823B1F08091E9008F7090917A
:1032E000EC0090FF02C090E801C090E0C92FC82B0D
:1032F0001092E9008091E80083FD0E94FE17CF70D4
:10330000C093E900CF910895881F8827881F0895EA
:1033100091E0883F08F490E0892F0895982F907FDE
:10332000903B99F038F4903981F0903A71F09038F0
:10333000C9F40BC0903DA1F018F4903C99F410C072
:10334000903E19F0903F71F402C083E00895E82F99
:10335000E15FEF3038F4F0E0E15FFD4F80810895E8
:1033600082E0089580E008950F932F774F776F7074
:10337000606BDC01ED91FC91022F242F462F63E05E
:1033800070E009950F9108950F932F774F776F7025
:103390006069DC01ED91FC91022F242F462F63E040
:1033A00070E009950F9108950F932F774F776F7005
:1033B0006068DC01ED91FC91022F242F462F63E021
:1033C00070E009950F910895FC017383628308955D
:1033D000FC01738F628F0895FC01758F648F0895CF
:1033E000CF93DF93EC011DA21FA21EA2BC01685D5A
:1033F0007F4F40EC88519F4F0E942D1C1B821A82E8
:103400001D821C821F821E82198618861B861A86C0
:103410001D861C861F861E86198A188A1B8A1A8A90
:103420001D8A1C8A1F8A1E8A198E188E1B8E1A8E60
:103430001D8E1C8E1F8E1E8E19A218A2DF91CF9199
:103440000895CF92DF92FF920F931F93CF93DF9354
:103450001F92CDB7DEB7F62E6A018C0108511F4FBF
:1034600008C0F60161916F01C80149830E94341CB4
:1034700049818C2D841B8F15A0F30F90DF91CF9184
:103480001F910F91FF90DF90CF900895FC01718301
:1034900060830895FC0171A360A30895AF92BF9269
:1034A000CF92DF92EF92FF920F931F93CF93DF9310
:1034B00000D01F92CDB7DEB77C016B01142FB22E66
:1034C000A02EDC0195968C9195978430F1F45A9654
:1034D000ED91FC915B97309709F4D8C0CB0101972F
:1034E00063E070E00E943434DB01AA0FBB1FA60F1B
:1034F000B71F49832A830B834C2D4A1B9E012F5FE4
:103500003F4FBD01C7010995B1C06230710509F493
:1035100053C06330710529F06130710509F09CC01A
:1035200083C0842F807F803A01F130F48038B9F075
:10353000803909F0ABC00DC0803EE9F0803F09F151
:10354000803B09F0A3C0D7011296ED91FC9113972F
:1035500023C0D7011496ED91FC9115971DC0D7019A
:103560001696ED91FC91179717C0D7011896ED911B
:10357000FC91199711C0D7011A96ED91FC911B97F8
:103580000BC0423F09F082C0D7011C96ED91FC911F
:103590001D97309731F47AC0309709F477C0123F05
:1035A00021F42A2D4B2D62EF04C0612F6F702A2D5C
:1035B0004B2DC70109955AC0842F807F803D59F05B
:1035C000803F79F0803C09F061C0D7011E96ED91F3
:1035D000FC911F9719C0D7015096ED91FC9151971E
:1035E00013C0433F31F4D7015296ED91FC915397AC
:1035F00008C0413F09F04AC0D7015496ED91FC91B3
:103600005597309741F442C0309709F43FC0133FBB
:1036100011F0113F19F44B2D612F03C0612F6F7012
:103620004B2DC701099522C0842F0E948819882339
:1036300031F0D7015696ED91FC91579707C0163F90
:1036400029F5D7015896ED91FC9159973097F1F0F3
:10365000612FC70109950AC064307105A8F416C02E
:103660000A2D2B2D412FB601C7010995D7015E9672
:10367000ED91FC915F97309789F00A2D2B2D412F0A
:10368000B601C70109950AC0C12CD12CD7015C969F
:10369000ED91FC915D97309719F7E8CF0F900F905F
:1036A0000F90DF91CF911F910F91FF90EF90DF90DE
:1036B000CF90BF90AF900895EF92FF920F931F931A
:1036C000CF93DF93EC01162F862F0E948819882351
:1036D00069F0FDA081E08DA300E020E0412F61E0D2
:1036E00070E0CE010E944E1AFDA27CC0812F0E9484
:1036F00084194DA1882309F440C0443029F01AA34D
:1037000021E030E03FA32EA3812F0E948E1981304B
:1037100031F070F0823051F0833059F507C08DA33D
:1037200000E020E0412F61E070E01EC08DA35AC090
:10373000103F19F0173FE9F404C084E08DA31AA3E9
:103740003FC02EA13FA1C90163E070E00E94343464
:103750008C0F9D1FFC0112A3B9016F5F7F4F7FA3E8
:103760006EA30CA12BA14AA1CE010E944E1A1DA24C
:1037700039C01DA21FA21EA235C0442399F12EA15B
:103780003FA1C90163E070E00E9434347C01FE0176
:10379000E80FF91F12A3B9016F5F7F4F7FA36EA3DC
:1037A0008130910591F082E0E816F104D9F40CA182
:1037B0002BA14AA1CE010E944E1A8DA1843091F016
:1037C00081E090E09FA38EA30DC0423059F400E049
:1037D0002BA14AA1CE010E944E1A8DA1843011F076
:1037E000FFA2EEA2DF91CF911F910F91FF90EF907A
:1037F0000895CF92DF92EF92FF920F931F93CF9392
:10380000DF93EC01E8A1F9A1309709F009958E0149
:1038100008511F4FC8010E94661CE12CF12CC82ED4
:10382000D12C0FC060E0C8010E947A1C682FCE0125
:103830000E945C1B61E0C8010E948B1C8FEFE81A9C
:10384000F80AEC14FD0470F3DF91CF911F910F91F2
:10385000FF90EF90DF90CF900895FC014283748336
:1038600063831182108208950F931F93CF93DF9388
:10387000EC01062F0E94AC1C182F298130E0C901F1
:1038800001966A8170E00E944834488150E08417B4
:10389000950729F4812F0E94AF1C80E012C0EB81B4
:1038A000FC81E20FF31F00832981822F90E00196B3
:1038B0006A8170E00E9448348983812F0E94AF1C86
:1038C00081E0DF91CF911F910F910895CF93DF9306
:1038D000EC010E94AC1C29819881291710F0C22F9D
:1038E00002C0CA81C20FC91B0E94AF1C8C2FDF917E
:1038F000CF910895FC012081862F90E0820F911DC9
:10390000628170E00E9448340380F481E02DE80F6A
:10391000F91F808108950F931F93CF93DF931F9218
:10392000CDB7DEB78C0169830E94AC1C482FF8012B
:1039300080816981262F30E0280F311D6281C90105
:1039400070E00E9448348083842F0F90DF91CF91E4
:103950001F910F910C94AF1C8FB7F89408958FBFEF
:103960000895FC01CB012091FA032430B1F42181A8
:103970002F702093E90040E050E064E070E00E9486
:103980007E1481110BC09091E80095FD07C09091C5
:10399000E8009E779093E800089582E008952091D2
:1039A000FA032430A9F4FC0181818F708093E9002F
:1039B0003091F3002091F200932F80E0822B892B2D
:1039C00049F08091E8008E778093E8000C943B16D4
:1039D00082E0089580E008952091FA03243051F4A4
:1039E000FC0121812F702093E9002091E80020FD47
:1039F0000C94CF1C0895FC01CB012091FA032430D4
:103A000011F080E0089526812F702093E900209125
:103A1000E80022FFF6CF2091E80025FFF2CF40E03A
:103A200050E064E070E00E94CD148091E80085FDD4
:103A300005C08091E8008B778093E80081E00895CD
:103A400090939502809394020895E0919402F091EE
:103A50009502309721F00190F081E02D099480E0EB
:103A60000895E0919402F0919502309721F0028040
:103A7000F381E02D09940895E0919402F09195026C
:103A8000309721F00480F581E02D0994089520916C
:103A90009602309197028217930771F090939702E4
:103AA00080939602E0919402F0919502309721F074
:103AB0000680F781E02D09940895209198023091B5
:103AC00099028217930771F090939902809398025C
:103AD000E0919402F0919502309721F00084F185F5
:103AE000E02D0994089508950C94731D0E94952962
:103AF0000E94AD060E94692A0C9411300C94E705CF
:103B00005F926F927F928F929F92AF92BF92CF926D
:103B1000DF92EF92FF920F931F93CF93DF93CDB776
:103B2000DEB72A970FB6F894DEBF0FBECDBF0E9456
:103B3000BD079AE9C92E92E0D92E00E010E0AA2430
:103B4000A394B12C502E802F0E9411093C01F60144
:103B5000E190F1906F01E826F926E114F10431F4C7
:103B60000F5F1F4F0530110569F73AC08091F002D1
:103B700081FD0E941A0920E030E04501022E02C0BA
:103B8000880C991C0A94E2F7C4018E219F21892B8D
:103B900009F12E835F826820792081E0672809F48B
:103BA00080E088870E949E298160782F9A87898784
:103BB0004E815F8168858A850E94391EF801EE0F6B
:103BC000FF1FE656FD4F80819181882599259183BD
:103BD000808316C02F5F3F4F2C30310571F6C0CF68
:103BE0008FEF89838A831B820E949E298160782FB0
:103BF0009D838C8349815A816B818D810E94391EFE
:103C00000E94562D1091A4020E94251D1817D9F06C
:103C10000E94251D8093A4022A960FB6F894DEBF59
:103C20000FBECDBFDF91CF911F910F91FF90EF900D
:103C3000DF90CF90BF90AF909F908F907F906F90CC
:103C40005F900C947E1D2A960FB6F894DEBF0FBECF
:103C5000CDBFDF91CF911F910F91FF90EF90DF903B
:103C6000CF90BF90AF909F908F907F906F905F901C
:103C70000895CF93DF93CDB7DEB72B970FB6F894A7
:103C8000DEBF0FBECDBF4F83588769877A878B878A
:103C9000DE01119686E0FD0111928A95E9F785E033
:103CA000FE01379601900D928A95E1F749815A817C
:103CB0006B817C818D819E810E9415262B960FB68B
:103CC000F894DEBF0FBECDBFDF91CF910895CF93A3
:103CD000C82F882309F4C1C0823859F40E94251DD9
:103CE00081FDBBC089E30E947C280E94F82889E3FB
:103CF0000CC0833879F40E94251D80FDAEC083E599
:103D00000E947C280E94F82883E50E949E28CF917B
:103D10000C94F828843859F40E94251D82FD9DC01A
:103D200087E40E947C280E94F82887E4EECF845024
:103D3000813A48F48C2F0E94732F81118EC08C2FF2
:103D40000E947C28E4CF8C2F805E883050F4C770AE
:103D500081E090E001C0880FCA95EAF70E94BF2871
:103D6000D6CF8C2F855A833078F4C53A29F0C63ADD
:103D700031F482E890E005C081E890E002C083E879
:103D800090E0CF910C94471D8C2F885A833108F016
:103D900064C0C83A39F1C93A41F1CA3A49F1CB3A5B
:103DA00051F1CC3A59F1CD3A61F1C03B69F1CE3ACB
:103DB00071F1CF3A79F1C13B81F1C23B89F1C33B4B
:103DC00091F1C43B99F1C53BA1F1C63BA9F1C73BB9
:103DD000B1F1C83BB9F1C93BC1F1CA3BC9F58AE2AF
:103DE00092E038C082EE90E035C089EE90E032C0BB
:103DF0008AEE90E02FC085EB90E02CC086EB90E03F
:103E000029C087EB90E026C08CEC90E023C08DECBD
:103E100090E020C083E891E01DC08AE891E01AC0DC
:103E200082E991E017C084E991E014C081E292E058
:103E300011C083E292E00EC084E292E00BC085E202
:103E400092E008C086E292E005C087E292E002C0FC
:103E500080E090E0CF910C945D1DCF910895882370
:103E600009F44DC0823859F40E94251D81FF47C0D6
:103E700089E30E947C280E94F82889E30CC08338DB
:103E800071F40E94251D80FF3AC083E50E947C28C2
:103E90000E94F82883E50E949E280C94F828843814
:103EA00059F40E94251D82FF2AC087E40E947C28C5
:103EB0000E94F82887E4EFCF982F9450913A08F4A5
:103EC000EACF982F905E983058F4282F277081E021
:103ED00090E001C0880F2A95EAF70E94C528DDCF3F
:103EE000982F955A933020F480E090E00C94471D71
:103EF000885A833120F480E090E00C945D1D089591
:103F0000882321F00E94BF280C94F8280895882364
:103F100021F00E94C5280C94F8280895BF92CF92F2
:103F2000DF92EF92FF920F931F93CF93DF93CDB762
:103F3000DEB727970FB6F894DEBF0FBECDBF8C015A
:103F400085E0F801DE01119601900D928A95E1F766
:103F5000F80130812181F280558152955F70838113
:103F60009481892B39F02F3F41F481E090E03F3F6D
:103F700031F003C081E090E002C080E090E080FD7D
:103F800073C339832A8389819A815E830E94392889
:103F9000B92E8F830E9438280E9460272B2D2295EE
:103FA0002F7030E05E816F812530310509F4E6C065
:103FB0006CF4243031050CF0A2C04B2D407F8B2DCA
:103FC0008F70223031050CF045C017C02C30310500
:103FD0004CF42A3031050CF0E7C12830310509F0E6
:103FE00043C3E5C02D30310509F4BAC20CF4A2C2B6
:103FF0002F30310509F038C323C3182F411101C0F8
:1040000002C01295107FFF2059F0112309F46BC2F2
:10401000812F6F830E94CF280E94F8286F8163C28E
:10402000862F0E942F1F112309F41EC3812F0E9487
:10403000D52827960FB6F894DEBF0FBECDBFDF910F
:10404000CF911F910F91FF90EF90DF90CF90BF9095
:104050000C94F828403211F08295807F662319F085
:10406000613071F523C0FF20B1F0511101C032C0A1
:10407000513081F527960FB6F894DEBF0FBECDBF45
:10408000DF91CF911F910F91FF90EF90DF90CF9034
:10409000BF900C94DF28511101C003C0513009F4C6
:1040A000E3C28E830E94E2288E819AC1FF2021F014
:1040B000563008F0D9C20EC0553008F0D5C290C1B4
:1040C000FF20C9F0552331F0F801958190FF0BC214
:1040D0009F70958327960FB6F894DEBF0FBECDBFB5
:1040E000DF91CF911F910F91FF90EF90DF90CF90D4
:1040F000BF900C94801F552309F472C109C22B2D67
:1041000026952695237030E02115310529F02130C0
:10411000310509F0A9C219C0FF2021F0862F9B2D7F
:10412000937002C080E090E027960FB6F894DEBF4F
:104130000FBECDBFDF91CF911F910F91FF90EF90F8
:10414000DF90CF90BF900C94471DFF2021F0862F69
:104150009B2D937002C080E090E027960FB6F894F4
:10416000DEBF0FBECDBFDF91CF911F910F91FF90AA
:10417000EF90DF90CF90BF900C945D1D862FFF20B5
:1041800019F00E945C2C02C00E94C42C27960FB626
:10419000F894DEBF0FBECDBFDF91CF911F910F917D
:1041A000FF90EF90DF90CF90BF900C944B2D8B2D14
:1041B000837009F079C0F11057C2262F22952695F9
:1041C0002770220F220F862F8F70C82ED12CE12C42
:1041D000F12C022E04C0CC0CDD1CEE1CFF1C0A943A
:1041E000D2F764FF10C06FE070E080E090E004C0A0
:1041F000660F771F881F991F2A95D2F760957095D3
:104200008095909503C060E070E0CB012B2D269542
:1042100026952370422F50E042305105D9F04330AB
:10422000510569F16C297D298E299F29413051055D
:1042300051F127960FB6F894DEBF0FBECDBFDF91C8
:10424000CF911F910F91FF90EF90DF90CF90BF9093
:104250000C9475276C297D298E299F2927960FB6E6
:10426000F894DEBF0FBECDBFDF91CF911F910F91AC
:10427000FF90EF90DF90CF90BF900C9487270E9423
:104280007527C701B60127960FB6F894DEBF0FBE9B
:10429000CDBFDF91CF911F910F91FF90EF90DF90F5
:1042A000CF90BF900C946327FF2019F08B2D817065
:1042B00001C08695882309F4D7C1262F229526951B
:1042C0002770220F220F862F8F70C82ED12CE12C41
:1042D000F12C022E04C0CC0CDD1CEE1CFF1C0A9439
:1042E000D2F764FF10C06FE070E080E090E004C09F
:1042F000660F771F881F991F2A95D2F760957095D2
:104300008095909503C060E070E0CB012B2D269541
:1043100026952370422F50E042305105D9F04330AA
:10432000510569F16C297D298E299F29413051055C
:1043300051F127960FB6F894DEBF0FBECDBFDF91C7
:10434000CF911F910F91FF90EF90DF90CF90BF9092
:104350000C9414286C297D298E299F2927960FB645
:10436000F894DEBF0FBECDBFDF91CF911F910F91AB
:10437000FF90EF90DF90CF90BF900C9426280E9482
:104380001428C701B60127960FB6F894DEBF0FBEFA
:10439000CDBFDF91CF911F910F91FF90EF90DF90F4
:1043A000CF90BF900C940228603F59F120F4603EFA
:1043B00008F494C008C0623F09F467C0F0F1633F9D
:1043C00009F08CC065C0162F1F708B2D8F71FF20D8
:1043D00021F00E94AD27812F7DCE0E94C827812F1A
:1043E00027960FB6F894DEBF0FBECDBFDF91CF91F9
:1043F0001F910F91FF90EF90DF90CF90BF900C94A2
:10440000871FFF20B1F0553008F02EC18B2D8F7122
:1044100027960FB6F894DEBF0FBECDBFDF91CF91C8
:104420001F910F91FF90EF90DF90CF90BF900C9471
:10443000E727563008F018C1E9CFFF2099F08B2DFF
:104440008F7127960FB6F894DEBF0FBECDBFDF91F8
:10445000CF911F910F91FF90EF90DF90CF90BF9081
:104460000C94AD278B2D8F7127960FB6F894DEBF75
:104470000FBECDBFDF91CF911F910F91FF90EF90B5
:10448000DF90CF90BF900C94C827F110EBCFD7CF1F
:10449000FF2099F08B2D8F7127960FB6F894DEBF11
:1044A0000FBECDBFDF91CF911F910F91FF90EF9085
:1044B000DF90CF90BF900C949E2727960FB6F8946C
:1044C000DEBF0FBECDBFDF91CF911F910F91FF9047
:1044D000EF90DF90CF90BF900C949927FF20A9F028
:1044E000552309F4ACCF862F27960FB6F894DEBF7C
:1044F0000FBECDBFDF91CF911F910F91FF90EF9035
:10450000DF90CF90BF900C94671E552309F4AACF7B
:10451000862F27960FB6F894DEBF0FBECDBFDF9172
:10452000CF911F910F91FF90EF90DF90CF90BF90B0
:104530000C942F1F4B2D4F70C8010E941A03279611
:104540000FB6F894DEBF0FBECDBFDF91CF911F91A4
:104550000F91FF90EF90DF90CF90BF900C94CB26FF
:10456000F11082C09B2D9F70492F50E042305105C1
:1045700099F144F44115510569F04130510509F0B4
:1045800073C019C043305105C1F14430510509F0E1
:104590006BC044C027960FB6F894DEBF0FBECDBFE8
:1045A000DF91CF911F910F91FF90EF90DF90CF900F
:1045B000BF900C94223027960FB6F894DEBF0FBE42
:1045C000CDBFDF91CF911F910F91FF90EF90DF90C2
:1045D000CF90BF900C94393027960FB6F894DEBF79
:1045E0000FBECDBFDF91CF911F910F91FF90EF9044
:1045F000DF90CF90BF900C94553027960FB6F8946B
:10460000DEBF0FBECDBFDF91CF911F910F91FF9005
:10461000EF90DF90CF90BF900C946830862F279654
:104620000FB6F894DEBF0FBECDBFDF91CF911F91C3
:104630000F91FF90EF90DF90CF90BF900C948C3053
:104640004B2D4F70C80127960FB6F894DEBF0FBEF2
:10465000CDBFDF91CF911F910F91FF90EF90DF9031
:10466000CF90BF900C941B0927960FB6F894DEBF2D
:104670000FBECDBFDF91CF911F910F91FF90EF90B3
:10468000DF90CF90BF9008950E94DC280E94B1284F
:104690000E94F8280E94F72D0E944B2D80E090E0A8
:1046A0000E94471D80E090E00C945D1D0E94CC2884
:1046B0000C9444230E943928292F22952F7030E032
:1046C0002C3031054CF42A3031056CF4225031097C
:1046D0002230310590F407C02C30310551F02F30D5
:1046E000310559F406C0803E10F0803F31F481E07E
:1046F000089593FB882780F9089580E00895CF936B
:10470000DF9300D000D01F92CDB7DEB70F900F908F
:104710000F900F900F90DF91CF910895CF93DF937B
:1047200000D000D000D0CDB7DEB726960FB6F894F3
:10473000DEBF0FBECDBFDF91CF9108951F93CF9302
:10474000DF93C091DB0216E012C0D0E01C9FF001A5
:104750001D9FF00D1124E555FD4F4081518162816F
:104760007381848195810E948E232196C7708091E8
:10477000DC02C813EACFDF91CF911F9108954091D9
:10478000A5025091A6026091A7027091A8028091A3
:10479000A9029091AA020C948E230F931F93CF939A
:1047A000DF938091AA0282958F7009F069C0809191
:1047B000A702882309F464C0A091DB02D091DC0237
:1047C000B091A502C091A6028091A8029091A90281
:1047D00021E030E0BF3F11F020E030E0122FBC01BB
:1047E0006095709506E04AC0009721F0CF3F29F40C
:1047F000212F05C021E030E002C020E030E020FDA4
:104800003BC04A2F50E0049FF001059FF00D11249A
:10481000E555FD4F2181C2132FC02081B2132CC05A
:104820002281211129C0238134812817390718F0EA
:10483000281B390B02C0260F371F283C3105E0F436
:104840008091AA028F7080618093AA0286E0849F83
:10485000F001859FF00D1124E055FD4F80818F7090
:104860008061808385EA92E00E948E1FDF91CF9164
:104870001F910F910C949E23AF5FA770AD13B4CF1F
:10488000DF91CF911F910F910895EF92FF920F93B7
:104890001F93CF93DF93CDB7DEB762970FB6F8942F
:1048A000DEBF0FBECDBF8C0185E0F801DE011D9695
:1048B00001900D928A95E1F7D8014C9111965C9187
:1048C000119712966C9112971396ED90FC90149795
:1048D0007091A502E091A6028091A8029091A90290
:1048E000009739F0EF3F41F421E030E07F3F31F0B5
:1048F00003C021E030E002C020E030E020FD5CC1D8
:104900002091A702222309F4F1C0E816F90628F045
:104910009701281B390BC90104C0809590958E0D15
:104920009F1D883C910508F098C08091AA02982F9D
:10493000907F09F064C0E51314C0741312C06111B4
:1049400010C08F7080618093AA020E94BF2385EA05
:1049500092E00E948E1F8091AA02D80115968C9336
:1049600043C1EF2839F05F3F41F481E090E04F3FD1
:1049700031F003C081E090E002C080E090E080FD73
:1049800003C081E0862702C080E090E080FF2EC057
:104990008091DB022091DC0236E013C090E0389F6A
:1049A000F001399FF00D1124E555FD4F718157132A
:1049B00006C07081471303C07281671317C0019648
:1049C00087708213EBCF12C19F7059F0882309F4CE
:1049D0000BC107C09F7029F0F8019581907F09F401
:1049E00003C1805E883008F4FFC0D2C0662309F49A
:1049F000FBC08091AA0281608093AA02F5C0E513F2
:104A000008C0741306C0611104C0D80115968C93B8
:104A10009DC04D875E878D859E856A8B0E945A2337
:104A20006A89882309F4B4C0662309F4B1C02091CF
:104A3000AA02822F82958F7090E002970CF4C6C074
:104A40008091A5029091A60298878F831986FB8694
:104A5000EA862C87CE01079646C08091AA02982F3D
:104A6000907F59F47E2DF98AE88A89890E947F23F4
:104A700085EA92E00E948E1F95C0E51311C0741361
:104A80000FC061110DC0F8018583C8010E948E1FFF
:104A9000E5EAF2E086E0DF011D928A95E9F7A2C01F
:104AA0004D875E878D859E856A8B0E945A236A8911
:104AB000882309F46DC0662309F46AC02091AA0214
:104AC000822F82958F7090E002970CF47FC08091C6
:104AD000A5029091A6029A8389831B82FD82EC82B3
:104AE0002E83CE0101960E948E1F70C0E816F90633
:104AF00028F09701281B390BC90104C080959095B7
:104B00008E0D9F1D883C910508F046C0662309F470
:104B10003FC0E51330C074132EC02091AA0220FDBF
:104B200021C0322F32953F70832F90E00097D1F053
:104B3000D80115962C9315970F9741F0832F8F5F0F
:104B40008295807F2F70282B15962C93C8010E9488
:104B50008E1F86E0F801A5EAB2E001900D928A95D9
:104B6000E1F73EC086E0F801A5EAB2E001900D92BF
:104B70008A95E1F737C04D875E878D859E850E94B7
:104B80005A23811123C08091AA0281608093AA02D6
:104B9000C8010E948E1F26C07E2DF98AE88A898965
:104BA0000E947F23E5EAF2E086E0DF011D928A950C
:104BB000E9F70E94BF2318C0662351F34D875E8733
:104BC0008D859E850E945A23882311F386E0F80183
:104BD000A5EAB2E001900D928A95E1F70E94CD23FB
:104BE0000E94BF2381E014C080E012C04D875E8721
:104BF0008D859E850E943928292F22952F7030E0BF
:104C0000223031050CF4E0CE243031050CF6E2CE32
:104C100062960FB6F894DEBF0FBECDBFDF91CF9185
:104C20001F910F91FF90EF9008951F93CF93DF9303
:104C3000CDB7DEB72C970FB6F894DEBF0FBECDBF51
:104C40004F83588769877A878B879C87CE01079621
:104C50000E9445248823D9F02F8138858A859B8539
:104C6000892B39F03F3F19F080E090E004C02F3FDE
:104C7000D9F781E090E0892B09F06DC04F8158850C
:104C800069857A858B859C850E948E2364C086E029
:104C9000FE013796DE01119601900D928A95E1F79B
:104CA000FF81E8854A855B854115510539F0EF3F65
:104CB00041F481E090E0FF3F31F003C081E090E0FB
:104CC00002C080E090E080FD46C02091DC0230E030
:104CD000C9010196877099276091DB0270E0861701
:104CE000970709F440C0F983EA835D834C8396E01B
:104CF000929FD001939FB00D1124A555BD4FFE0189
:104D0000319601900D929A95E1F78093DC020E9412
:104D10009E2321C0189FC001112485559D4F0E94DC
:104D20004524882371F1E091DB021E9FF0011124DC
:104D3000E555FD4F40815181628173818481958168
:104D40000E948E238091DB0290E001968770992764
:104D50008093DB0201C016E08091DB029091DC02BF
:104D60008913D8CF0EC00E9456231092DC021092F5
:104D7000DB02E5EAF2E086E0DF011D928A95E9F7C1
:104D8000EACF2C960FB6F894DEBF0FBECDBFDF91F1
:104D9000CF911F910895DF92EF92FF920F931F938F
:104DA000CF93DF93EC01009709F46EC0D12CEE2471
:104DB000E394F12C8E010F5F1F4FFE018491843725
:104DC00048F4843008F04CC0813071F0823009F032
:104DD0005BC01EC0853709F43FC080F1982F9458FE
:104DE000903708F051C03FC02296F8018491982F67
:104DF000905E983050F48770FE2D01C0FF0F8A95A9
:104E0000EAF78F2F0E94CF2813C00E94671E2FC081
:104E10002296F8018491982F905E983060F4877004
:104E2000FE2D01C0FF0F8A95EAF78F2F0E94D5282B
:104E30000E94F8281CC00E942F1F19C02296F8015A
:104E4000049107C08FE99FE00197F1F700C00000CF
:104E500001500111F7CF0BC02296F801D49007C082
:104E60000E94671E03C08F770E942F1FE8018D2DBF
:104E700007C08150EFE9FFE03197F1F700C0000073
:104E8000882309F497CFF5CFDF91CF911F910F9130
:104E9000FF90EF90DF9008956093E1027093E2023B
:104EA0008093E3029093E4020C9444236093DD0228
:104EB0007093DE028093DF029093E0020C9444230F
:104EC00008950C944C270F931F930091E1021091C9
:104ED000E2022091E3023091E402602B712B822BDD
:104EE000932B1F910F910C944C270F931F930091BC
:104EF000E1021091E2022091E3023091E40260238A
:104F00007123822393231F910F910C944C270F93AD
:104F10001F930091E1021091E2022091E30230918F
:104F2000E40260277127822793271F910F910C9429
:104F30004C2760E070E0CB010C94562741E050E034
:104F400060E070E004C0440F551F661F771F8A950C
:104F5000D2F7CB01BA010C94562741E050E060E053
:104F600070E004C0440F551F661F771F8A95D2F763
:104F70008091DD029091DE02A091DF02B091E0020B
:104F8000482B592B6A2B7B2BCB01BA010C9456274B
:104F900041E050E060E070E004C0440F551F661F20
:104FA000771F8A95D2F740955095609570958091BE
:104FB000DD029091DE02A091DF02B091E002482371
:104FC00059236A237B23CB01BA010C94562741E075
:104FD00050E060E070E004C0440F551F661F771F6B
:104FE0008A95D2F78091DD029091DE02A091DF02D6
:104FF000B091E002482759276A277B27CB01BA01E5
:105000000C9456270F931F930091DD021091DE023E
:105010002091DF023091E002602B712B822B932BC9
:105020001F910F910C9456270F931F930091DD024F
:105030001091DE022091DF023091E00260237123A3
:10504000822393231F910F910C9456270F931F9344
:105050000091DD021091DE022091DF023091E0022A
:1050600060277127822793271F910F910C94562751
:105070000895CF92DF92EF92FF920F931F93CF93F9
:10508000DF93EC01C090E102D090E202E090E302F5
:10509000F090E4028091DD029091DE02A091DF02A7
:1050A000B091E002C82AD92AEA2AFB2A0FE110E0CF
:1050B000B701A601002E04C07695679557954795D0
:1050C0000A94D2F740FF08C0BE01802F0E947104ED
:1050D0008130910509F007C00150110948F7BE0160
:1050E00080E00E947104DF91CF911F910F91FF909A
:1050F000EF90DF90CF90089540918B0150918C01FB
:1051000020E030E09FEFFA01E20FF31F62816817A1
:10511000A1F09F3F19F4611101C0922F2F5F3F4F03
:105120002630310581F707C0FA01E90FF11D97FD1F
:10513000FA95828308959F3FB9F7089540918B01B6
:1051400050918C0120E030E0FA01E20FF31F9281D0
:10515000981301C012822F5F3F4F26303105A1F70F
:10516000089581E090E0E0918B01F0918C01E80FCF
:10517000F91F1082019688309105A9F70895909142
:10518000E502982B9093E502089580959091E502B1
:1051900098239093E50208951092E5020895909166
:1051A000E602982B9093E602089580959091E6028E
:1051B00098239093E60208951092E6020895809352
:1051C000E70208951092E702089540918B015091F3
:1051D0008C0120E030E080E0FA01E20FF31F9181C2
:1051E00091118F5F2F5F3F4F27303105A9F7089549
:1051F000E0918B01F0918C018091E5028083E09138
:105200008B01F0918C0180819091E602892B808343
:105210009091E702992361F0E0918B01F0918C016C
:105220008081892B80830E94E52881110E94E228D9
:1052300080918B0190918C010C94311D8091FA0327
:10524000843021F11092F10220E488E190E00FB661
:10525000F894A895809360000FBE2093600080E0D2
:105260000E94590383B7817F846083BF83B78160C5
:1052700083BF7894889583B78E7F83BF88E10FB60C
:10528000F89480936000109260000FBE0895089516
:105290000895CF9380E00E9459030E9447290E94FD
:1052A000BD070E944829C0E08C2F0E941109892B5C
:1052B00029F4CF5FC530C1F780E001C081E0CF9114
:1052C00008950E94562380E00E9459030E941130E5
:1052D0000E94251D0C94E7051F920F920FB60F92A6
:1052E00011248F939F93AF93BF938091F10281110B
:1052F00013C08091F2029091F302A091F402B09158
:10530000F5024196A11DB11D8093F2029093F30224
:10531000A093F402B093F502BF91AF919F918F914A
:105320000F900FBE0F901F90189582E084BD93E000
:1053300095BD9AEF97BD80936E0008958FB7F8944E
:105340004091F2025091F3026091F4027091F502E3
:105350008FBFCA010895CF92DF92EF92FF920F9311
:105360001F932FB7F8944091F2025091F30260918D
:10537000F4027091F5022FBF6A017B01EE24FF2435
:105380008C0120E030E0C016D106E206F30620F0E2
:105390009A01281B390B05C09C0120953095240FDC
:1053A000351FC9011F910F91FF90EF90DF90CF90B3
:1053B00008951F920F920FB60F9211248F939F930F
:1053C000AF93BF938091F2029091F302A091F40207
:1053D000B091F5020196A11DB11D8093F202909348
:1053E000F302A093F402B093F502BF91AF919F91A5
:1053F0008F910F900FBE0F901F9018950E946D1601
:10540000F8942FEF87EA91E6215080409040E1F731
:1054100000C0000087E090EBDC01809304049093CF
:105420000504A0930604B09307042CE088E190E003
:105430000FB6F894A895809360000FBE209360008B
:10544000FFCFCF92DF92EF92FF920F931F93CF93F4
:10545000DF93C82ED12C01E010E08D2D0E941109A0
:105460007C01C0E0D0E098010C2E02C0220F331F57
:105470000A94E2F72E213F21232B29F42196CC30E8
:10548000D10589F708C06C2F7D2D80E00E944C0467
:10549000C812F4CF06C0D39485E0D812DECF80E0E6
:1054A00001C081E0DF91CF911F910F91FF90EF90AC
:1054B000DF90CF900895CF93C82F8CE20E94212ACD
:1054C000882321F08C2FCF910C94212A80E0CF915A
:1054D0000895CF930E94AC2B811102C00E948D2BA6
:1054E000C5E608C00E94BD078FE39CE90197F1F76C
:1054F00000C00000C150B1F789E20E945B2A81110F
:105500000AC18AE20E945B2A81110E948D2B85E0EC
:105510000E945B2A81110E94FE290E94B72B809372
:10552000F00287E00E945B2A882399F18BE10E94B8
:105530005B2A882351F09091F00291FB882780F933
:1055400021E0822780FB91F922C08EE00E945B2A35
:10555000882351F09091F00292FB882780F921E096
:10556000822780FB92F913C080E10E945B2A909110
:10557000F002882341F093FB882780F921E08227FD
:1055800080FB93F904C0892F809580FB90F990935C
:10559000F0028091F0020E94BB2B0E94C92B8093E5
:1055A000010380EE0E945B2A882341F08091010371
:1055B000982F909590FB80F98093010389E30E94D6
:1055C0005B2A882359F09091010391FB882780F989
:1055D00021E0822780FB91F99093010382EE0E94E3
:1055E0005B2A882359F09091010392FB882780F968
:1055F00021E0822780FB92F99093010386EE0E94BE
:105600005B2A882359F09091010393FB882780F946
:1056100021E0822780FB93F99093010383EE0E949F
:105620005B2A882359F09091010394FB882780F925
:1056300021E0822780FB94F99093010385E30E9487
:105640005B2A882359F09091010395FB882780F904
:1056500021E0822780FB95F99093010381E30E946A
:105660005B2A882359F09091010396FB882780F9E3
:1056700021E0822780FB96F99093010381E10E944B
:105680005B2A882359F09091010397FB882780F9C2
:1056900021E0822780FB97F9909301038091010319
:1056A0000E94CD2B87E20E945B2AC82F8EE10E94C8
:1056B0005B2A8111C2608FE10E945B2A8111C46064
:1056C00080E20E945B2A8111C86081E20E945B2A0D
:1056D0008111C06182E20E945B2A8111C06283E273
:1056E0000E945B2A8111C06484E20E945B2A8823A5
:1056F00011F0C06802C0CC2329F08C2F0E94C42B6B
:105700006C2F03C00E94C02B682F70E080E090E0F7
:10571000CF910C946127CF9108956DEE7EEF80E0DC
:1057200090E00E94783460E082E090E00E946A3469
:1057300060E083E090E00E946A3460E084E090E002
:105740000E946A3460E085E090E00E946A3460E084
:1057500086E090E00C946A3480E090E00E9464342B
:1057600021E08D3E9E4F09F020E0822F089582E0D7
:1057700090E00C945C34682F82E090E00C946A34E2
:1057800083E090E00C945C34682F83E090E00C940C
:105790006A3484E090E00C945C34682F84E090E0FC
:1057A0000C946A3486E090E00C945C34682F86E0B8
:1057B00090E00C946A348091FE0280FF0BC06091EF
:1057C000900185E0689FB0011124759567957595E6
:1057D00067952AC081FF09C06091900185E0689FAC
:1057E000B0011124759567951FC082FF07C06091B5
:1057F000900185E0689FB001112416C04091F80225
:105800004423C9F060918F01461788F720919001D9
:1058100085E0289F90011124429FC001439F900D75
:10582000112470E00E9448346038710540F461151D
:10583000710539F002C065E070E0862F08958FE7AA
:10584000089581E008958091FE0280FF08C0609174
:105850008E0170E0759567957595679521C081FFFC
:1058600006C060918E0170E07595679519C082FF42
:1058700004C060918E0170E010C08091F80288230E
:10588000C1F060918D018617A0F790918E01989FCD
:10589000C001112470E00E9448346038710528F47A
:1058A0006115710521F0862F08958FE7089581E035
:1058B000089561E070E0F4CF803F21F40E94DB2B7B
:1058C000819504C0813F29F40E94DB2B8093FB0269
:1058D0000895823F21F40E94DB2B819504C0833F11
:1058E00029F40E94DB2B8093FA020895893F19F472
:1058F0000E94232C05C08A3F31F40E94232C8195FD
:105900008093FC0208958B3F21F40E94232C819503
:1059100004C08C3F29F40E94232C8093FD0208953B
:10592000843F21F48091F902816017C0853F21F402
:105930008091F902826011C0863F21F48091F902C2
:1059400084600BC0873F21F48091F902886005C014
:10595000883F31F48091F90280618093F9020895C3
:105960008D3F21F48091FE0281600BC08E3F21F4B7
:105970008091FE02826005C08F3F29F48091FE0273
:1059800084608093FE020895803F29F48091FB0299
:1059900087FF6EC007C0813F41F48091FB0218165B
:1059A0000CF066C01092FB0263C09091FA02823F35
:1059B00019F497FF5DC005C0833F31F419160CF050
:1059C00057C01092FA0254C0893F31F48091FC0212
:1059D00018160CF04DC006C08A3F39F48091FC02C5
:1059E00087FF46C01092FC0243C08B3F29F4809190
:1059F000FD0287FF3DC006C08C3F39F48091FD0257
:105A00001816B4F51092FD0233C0843F21F4809142
:105A1000F9028E7F05C0853F31F48091F9028D7FB8
:105A20008093F90225C0863F21F48091F9028B7F93
:105A3000F7CF873F21F48091F902877FF1CF883F2C
:105A400021F48091F9028F7EEBCF8D3F21F480917C
:105A5000FE028E7F0BC08E3F21F48091FE028D7F6F
:105A600005C08F3F29F48091FE028B7F8093FE0258
:105A70008091FA0281110EC08091FB0281110AC04F
:105A80008091FC02811106C08091FD02811102C04B
:105A90001092F802089589EF92E00E943C1D0E9446
:105AA0009E299093F7028093F6020895CF938091F8
:105AB000F6029091F7020E94AB294091F80244232C
:105AC00021F02091910130E006C0209192015AE02E
:105AD000259F900111248217930708F486C08091B6
:105AE000FA0281110DC09091FB02911109C09091B1
:105AF000FC02911105C09091FD02992309F475C033
:105B00004F3F19F04F5F4093F802181624F40E949B
:105B1000DB2B8093FA028091FA0287FF05C00E9476
:105B2000DB2B81958093FA028091FB02181624F4F6
:105B30000E94DB2B8093FB028091FB0287FF05C054
:105B40000E94DB2B81958093FB026091FA02662311
:105B500039F1C091FB02CC2319F1772767FD7095CD
:105B6000872F972F0E94AC3123E333E343E35FE3B6
:105B70000E9460320E9479316093FA026C2F77277D
:105B800067FD7095872F972F0E94AC3123E333E395
:105B900043E35FE30E9460320E9479316093FB022D
:105BA0008091FC02181624F40E94232C8093FC029E
:105BB0008091FC0287FF05C00E94232C8195809371
:105BC000FC028091FD02181624F40E94232C80937D
:105BD000FD028091FD0287FF05C00E94232C819564
:105BE0008093FD02CF910C944B2DCF910895E9EF56
:105BF000F2E085E0DF011D928A95E9F71092F80244
:105C00001092FE020895833089F130F4813061F002
:105C1000823009F06EC019C0853009F449C0B8F16E
:105C2000863009F066C055C020919201862F90E021
:105C3000820F911D8F3F910520F4620F60939201B6
:105C400008958FEF80939201089520919101862FFE
:105C500090E0820F911D8F3F910520F4620F6093B9
:105C6000910108958FEF8093910108952091900103
:105C7000862F90E0820F911D8F3F910520F4620FD7
:105C80006093900108958FEF809390010895209183
:105C90008F01862F90E0820F911D8F3F910520F498
:105CA000620F60938F0108958FEF80938F010895A5
:105CB00020918E01862F90E0820F911D8F3F9105DC
:105CC00020F4620F60938E0108958FEF80938E0110
:105CD000089520918D01862F90E0820F911D8F3FB6
:105CE000910520F4620F60938D0108958FEF8093EA
:105CF0008D010895833021F130F4813059F08230E4
:105D000009F049C012C0853089F128F1863009F0C8
:105D100042C037C080919201681720F4861B80939F
:105D2000920108951092920108958091910168174F
:105D300020F4861B8093910108951092910108959B
:105D400080919001681720F4861B8093900108953C
:105D500010929001089580918F01681720F4861B9E
:105D600080938F01089510928F01089580918E0184
:105D7000681720F4861B80938E01089510928E017F
:105D8000089580918D01681720F4861B80938D0102
:105D9000089510928D01089541E050E060E070E0B8
:105DA00004C0440F551F661F771F8A95D2F7CB0199
:105DB000BA010E9461270C945623873200F58E3178
:105DC00008F086C08E3009F466C060F4873009F4AC
:105DD0004DC018F4863049F531C0883041F18B3020
:105DE00021F57BC0863109F478C018F48031E9F4DC
:105DF0005CC0893109F471C08B31B9F442C0883379
:105E000009F46BC048F4893209F460C0853309F4A1
:105E10005DC0873251F45AC0833409F457C018F476
:105E20008A3318F057C0883499F080E008950E94B2
:105E3000B72B0E94C92B0E94D22B4FC08091F00239
:105E4000817F8E7F8093F00281E08093FF0208952E
:105E50000E9456232FEF83ED90E321508040904025
:105E6000E1F700C000000E94FE2937C08091F002D7
:105E700080FF03C0817F8E7F01C081608093F0022C
:105E80002CC09091F00291FB882780F921E08227B5
:105E900080FB91F913C09091F00292FB882780F962
:105EA00021E0822780FB92F909C09091F00293FBD8
:105EB000882780F921E0822780FB93F99093F002F4
:105EC000882359F091609093F00207C080E003C0EE
:105ED0008D5101C089530E94CC2E81E0089580E04D
:105EE000089580E00895CF93C82F8091FF028130FC
:105EF00071F020F0823009F089C037C0A0918B0189
:105F0000B0918C018C91823209F082C007C0A091BF
:105F10008B01B0918C018C91823249F48C2F0E94BC
:105F20006F2F81111EC08C2F0E94DD2E1CC08C2F64
:105F30000E94712F811115C0C43169F030F4CB304B
:105F400081F0C03109F068C009C0C93221F0C833FE
:105F500009F062C006C01092FF025EC082E080932A
:105F6000FF0281E090E081705AC0C932C9F060F44C
:105F7000C431B1F020F4C73009F04CC034C0CE5168
:105F8000C63008F047C017C0CE3439F120F4CB3406
:105F900009F040C01CC0C135C1F0C235D9F513C0ED
:105FA00080910003882319F01092000333C081E030
:105FB0008093FF0234C0EC2FF0E0E25EFD4F808161
:105FC0008093000327C061E003C061E007C06AE07E
:105FD000809100030E94032E1DC06AE0809100039F
:105FE0000E947A2E17C08EE18093920182E3809303
:105FF00091018AE08093900184E180938F0188E091
:1060000080938E0188E280938D0104C01092FF027C
:1060100080E005C081E003C080E090E0A4CFCF9194
:1060200008950E94AC2B811102C00E948D2B0E940A
:10603000D22B8093030480FF02C0869501C080E0CC
:106040000C94590380910304982F9695292F30E0E2
:10605000233031054CF49F5F990F8170892B81604B
:10606000809303040E94D62B8091030486950C94A0
:10607000590380910304982F969591F09158990FA8
:106080008170892B809303048E7F91E009F490E066
:106090008091030490FB80F9809303040E94D62B27
:1060A0008091030486950C94590380910304982FE2
:1060B000909590FB80F9809303040E94D62B8091E9
:1060C000030480FF02C0869501C080E00C94590350
:1060D00030910304232F26952F5F2F77822F90E096
:1060E000317004972CF4220F232B2093030402C059
:1060F0003093030480910304282F2E7F91E009F44C
:1061000090E090FB80F9809303040E94D62B80914D
:10611000030486950C94590320910304922F9695BD
:106120009827990F822F8170892B809303048E7F8B
:1061300091E009F490E08091030490FB80F9809352
:1061400003040E94D62B8091030486950C94590376
:106150005058BB27AA270ED075C166D130F06BD13D
:1061600020F031F49F3F11F41EF45BC10EF4E09572
:10617000E7FB51C1E92F77D180F3BA1762077307A4
:106180008407950718F071F49EF58FC10EF4E09521
:106190000B2EBA2FA02D0B01B90190010C01CA01E1
:1061A000A0011124FF27591B99F0593F50F4503E8C
:1061B00068F11A16F040A22F232F342F4427585F7E
:1061C000F3CF469537952795A795F0405395C9F796
:1061D0007EF41F16BA0B620B730B840BBAF091504E
:1061E000A1F0FF0FBB1F661F771F881FC2F70EC0ED
:1061F000BA0F621F731F841F48F4879577956795C0
:10620000B795F7959E3F08F0B3CF9395880F08F0A8
:106210009927EE0F979587950895D9D008F481E0D6
:1062200008950CD00FC107D140F0FED030F021F41A
:106230005F3F19F0F0C0511139C1F3C014D198F388
:106240009923C9F35523B1F3951B550BBB27AA27F7
:1062500062177307840738F09F5F5F4F220F331F69
:10626000441FAA1FA9F333D00E2E3AF0E0E830D035
:1062700091505040E695001CCAF729D0FE2F27D038
:10628000660F771F881FBB1F261737074807AB0706
:10629000B0E809F0BB0B802DBF01FF2793585F4F7B
:1062A0002AF09E3F510568F0B6C000C15F3FECF395
:1062B000983EDCF3869577956795B795F7959F5F40
:1062C000C9F7880F911D9695879597F90895E1E094
:1062D000660F771F881FBB1F621773078407BA07F3
:1062E00020F0621B730B840BBA0BEE1F88F7E0954E
:1062F000089504D06894B111D9C00895BCD088F035
:106300009F5790F0B92F9927B751A0F0D1F0660FA1
:10631000771F881F991F1AF0BA95C9F712C0B130BC
:1063200081F0C3D0B1E00895C0C0672F782F8827CF
:10633000B85F39F0B93FCCF3869577956795B395FB
:10634000D9F73EF490958095709561957F4F8F4F6A
:106350009F4F0895E89409C097FB3EF4909580956F
:10636000709561957F4F8F4F9F4F9923A9F0F92F1B
:1063700096E9BB279395F695879577956795B79599
:10638000F111F8CFFAF4BB0F11F460FF1BC06F5F7F
:106390007F4F8F4F9F4F16C0882311F096E911C091
:1063A000772321F09EE8872F762F05C0662371F0B2
:1063B00096E8862F70E060E02AF09A95660F771FC6
:1063C000881FDAF7880F9695879597F90895990FA2
:1063D0000008550FAA0BE0E8FEEF16161706E807AF
:1063E000F907C0F012161306E407F50798F0621BD0
:1063F000730B840B950B39F40A2661F0232B242BA5
:10640000252B21F408950A2609F4A140A6958FEFC3
:10641000811D811D089597F99F6780E870E060E015
:1064200008959FEF80EC089500240A94161617062D
:1064300018060906089500240A9412161306140675
:1064400005060895092E0394000C11F4882352F0D8
:10645000BB0F40F4BF2B11F460FF04C06F5F7F4F90
:106460008F4F9F4F089557FD9058440F551F59F077
:106470005F3F71F04795880F97FB991F61F09F3F31
:1064800079F087950895121613061406551FF2CF5A
:106490004695F1DF08C0161617061806991FF1CFAA
:1064A00086957105610508940895E894BB276627D1
:1064B0007727CB0197F908958ADF08F48FEF0895C5
:1064C0000BD0C0CFB1DF28F0B6DF18F0952309F06C
:1064D000A2CFA7CF1124EACFC6DFA0F3959FD1F3B7
:1064E000950F50E0551F629FF001729FBB27F00D82
:1064F000B11D639FAA27F00DB11DAA1F649F6627D7
:10650000B00DA11D661F829F2227B00DA11D621F25
:10651000739FB00DA11D621F839FA00D611D221FDF
:10652000749F3327A00D611D231F849F600D211DC3
:10653000822F762F6A2F11249F5750408AF0E1F066
:1065400088234AF0EE0FFF1FBB1F661F771F881FAF
:1065500091505040A9F79E3F510570F05CCFA6CFF7
:106560005F3FECF3983EDCF3869577956795B7959A
:10657000F795E7959F5FC1F7FE2B880F911D9695C4
:10658000879597F90895FA01EE0FFF1F30962105C0
:10659000310599F16115710561F48038BFE39B07FE
:1065A00049F168949038810561F08038BFEF9B070E
:1065B00041F0992342F5FF3FE1053105210511F135
:1065C000E8940894E795D901AA2329F4AB2FBE2FAC
:1065D000F85FD0F310C0FF5F70F4A695E0F7F739CD
:1065E00050F019F0FF3A38F49F779F930CD00F903A
:1065F00007FC905808953EF014CF60E070E080E80A
:106600009FE308954FE79F775F934F933F932F93B7
:106610009ED02F913F914F915F9152DF05C019F4A9
:106620000EF0F9CE42CFFDCE26DFC8F39638C0F784
:1066300007F80F92E8942BE33AEA48EB5FE74EDF66
:106640000F920F920F924DB75EB70F92C0D0ECEA47
:10665000F0E016D04F915F91EF91FF91E595EE1F1D
:10666000FF1F49F0FE57E0684427EE0F441FFA95DC
:10667000E1F74195550B32D00F9007FE26C00895E3
:10668000DF93CF931F930F93FF92EF92DF927B01E3
:106690008C01689405C0DA2EEF011EDFFE01E8943C
:1066A000A5912591359145915591AEF3EF0162DDAC
:1066B000FE019701A801DA9479F7DF90EF90FF903F
:1066C0000F911F91CF91DF9108959B01AC0160E084
:1066D00070E080E89FE3A5CD9ECEACC0CCDEE8F3B1
:1066E0009923D9F3940F511DBBF39150504094F06E
:1066F00059F0882332F0660F771F881F9150504061
:10670000C1F79E3F510544F7880F911D96958795D7
:1067100097F908955F3FACF0983E9CF0BB278695B3
:1067200077956795B79508F4B1609395C1F7BB0F5E
:1067300058F711F460FFE8CF6F5F7F4F8F4F9F4F87
:10674000E3CFB4CE0EF076C06CCE689464CE93DE08
:10675000C8F39923D1F3C6F3DF93CF931F930F931D
:10676000FF92C92FDD2788232AF02197660F771F14
:10677000881FDAF720E030E040E85FEB9FE38839DC
:1067800020F0803E30F021968F77E3DCE4EDF0E0FE
:1067900003C0DFDCE1E0F1E073DF8B01BE01EC015F
:1067A000FB2E6F5771097595771F880B990BD4DDF8
:1067B00028E132E741E35FE38FDEAF2D9801AE01C0
:1067C000FF900F911F91CF91DF91D4DC3BCEFA0166
:1067D000DC01AA0FBB1F9B01AC01BF5728F4222785
:1067E0003327442750781FC0B75188F4AB2F0024BB
:1067F000469537952795011CA395D2F3002069F0A3
:10680000220F331F441FB395DAF30DD0A1CC6130B2
:106810007105A0E88A07B94630F49B01AC016627F0
:10682000772788279078309621F020833183428320
:10683000538308959F3F31F0915020F487957795C9
:106840006795B795880F911D9695879597F9089547
:10685000991B79E004C0991F961708F0961B881FB2
:106860007A95C9F780950895AA1BBB1B51E107C013
:10687000AA1FBB1FA617B70710F0A61BB70B881FD0
:10688000991F5A95A9F780959095BC01CD0108955F
:1068900097FB072E16F4009407D077FD09D00E94CD
:1068A000343407FC05D03EF4909581959F4F0895B0
:1068B000709561957F4F0895F999FECF92BD81BD86
:1068C000F89A992780B50895A8E1B0E042E050E039
:1068D0000C947F34262FF999FECF1FBA92BD81BD4B
:1068E00020BD0FB6F894FA9AF99A0FBE0196089552
:1068F0000E946A34272F0C946B34DC01CB01FC011D
:10690000F999FECF06C0F2BDE1BDF89A319600B408
:0E6910000D9241505040B8F70895F894FFCF13
:10691E0055D0A44600001644000000000000484276
:10692E0061978A460000C8430000000000004842FC
:10693E0055D024460000C843000000000000484225
:10694E0000005C460000C843000000000000484202
:10695E0061978A4600007A4455D0A4460000C84389
:10696E00000000000000484200005C460000C843E2
:10697E00000000000000484255D024460000164496
:10698E000507000C058540000001064000000100CF
:10699E0091102111FD10C810941001E8022808145E
:1069AE000A321E42004500250026004300610060A9
:1069BE000020003700640065006600670044004652
:1069CE000024004700000002000400050007000933
:1069DE00000B000C000E0010001100130015001724
:1069EE000018001A001C001D001F002100230024A7
:1069FE00002600280029002B002D002F0030003229
:106A0E000034003500370039003B00F6030F042830
:106A1E0004410469051C05E604C6043F4D362002F8
:106A2E000302000001000101010101000101010248
:086A3E00030405060708090026
:00000001FF
